:04000000A9EF1FF055
:1000080000C016F001C015F0E1CF17F0E2CF18F0EC
:10001800A4AA8FD0A3AA8DD0AACF7EF69CA202D084
:100028009C989C889CA404D0AACF7EF606017E6B7F
:100038000401F551000802E1F451FF0819E2F4C483
:100048007CF6F5C47DF6AACF7EF606017E6B0E0E11
:100058000401F425E16E050EF521E26EE66AF46B03
:10006800F56B010E06010E6F000E0F6FA39A61D09B
:1000780047D006017E51520A05E1010E0401196FAD
:10008800000E1A6F56D006017E514D0A05E1020E88
:100098000401196F000E1A6F4CD006017E51430AF5
:1000A80005E1030E0401196F000E1A6F240E0501F5
:1000B8000E6F470E0F6F500E106F520E116F4D0ED0
:1000C800126F430E136F050E0401F46F000EF56FE7
:1000D80030D00E0EF425E16E050EF521E26E7EC6D7
:1000E800E6FFF4C47CF6F5C47DF6010EF425006E37
:1000F800000EF521016E00C0F4F401C0F5F419D02A
:100108000401000E1A1902E1000E1919B2E0000EDE
:100118001A1902E1010E1919B6E0000E1A1902E1C6
:10012800020E1919BAE0000E1A1902E1030E191984
:10013800D0E0F2AA1ED0F2A41CD004016D0ED76E36
:10014800840ED66E010E525D006E000E5359016E7C
:1001580000C052F401C053F4800E5319006E800E93
:10016800005C02E1010E525D03E208014E83F29A3F
:10017800F2949EAA4AD09DAA48D0ACA203D0AC98CB
:10018800AC88AC92ACA402D0AFCFD7F6AFCFD7F63D
:100198000601D7510D0A0AE0000E006E08018951C8
:1001A800005C02E188513F0801E318D00801010E04
:1001B8004C6F000E4D6F9D9AEC0E8825E16E060E71
:1001C8008921E26EE66A88C8D5F689C8D6F6886BB2
:1001D800896BAFCFD7F60601D76B17D0EC0E0801A5
:1001E8008825E16E060E8921E26ED7C6E6FF88C82B
:1001F800D5F689C8D6F6010E8825006E000E89212D
:10020800016E00C088F801C089F816C000F015C05A
:0C02180001F017C0E1FF18C0E2FF110068
:0E022400ADB202D00000FCD7C7C8AEFF12007A
:080232000AAE029E000E12004C
:10023A000B840BAE28EF01F0010E036E026A016A0D
:0A024A00006A0A360232FF0E1200AD
:0E025400026A016A006A086A036A000E12005C
:100262000B820BAE3BEF01F0036802680168006885
:080272000A360232FF0E1200F1
:0E027A00A8B202D00000FCD7C7C8A9FF12002E
:10028800F250026EF29E0500FF6A0150FE6E0050A9
:08029800FD6E02BEF28E1200A1
:1002A00073B409D01F0E7114016E0150000A03E1EE
:0A02B000010E006E01D0006A12007A
:1002BA000CB09FEF01F00CA245EF02F00E6A000E9F
:1002CA000264B6EF01F0F00E0214D8A481EF01F037
:1002DA00023A01380F0B02260138F00B016E003882
:1002EA000F0B01260038F00B006E08380F0B0026A2
:1002FA000838F00B086E0E84D89002BE9AEF01F00F
:10030A0008360036013602360E2A02BE9AEF01F08E
:10031A0008360036013602360E2A02BE9AEF01F07E
:10032A0008360036013602360E2A0E5003643BEFB9
:10033A0002F0035E0BBC08AE40EF02F0D880800EDC
:10034A0008640030000E002201220222D8A040EFE9
:10035A0002F0023201320032034A45EF02F040EF66
:10036A0002F001C002F000C001F008C000F0086A03
:10037A00000E0E860264EDEF01F0F00E0214D8A40E
:10038A00D5EF01F0023A01380F0B02260138F00BC3
:10039A00016E00380F0B01260038F00B006E0E8438
:1003AA00D89002BE9AEF01F00036013602360E2AC4
:1003BA0002BE9AEF01F00036013602360E2A02BE5C
:1003CA009AEF01F00036013602360E2A9AEF01F052
:1003DA0001C002F000C001F0006A000E0E960E88FD
:1003EA0002641AEF02F0F00E0214D8A405EF02F02C
:1003FA00023A01380F0B02260138F00B016E0E8407
:10040A00D89002BE9AEF01F0013602360E2A02BED9
:10041A009AEF01F0013602360E2A02BE9AEF01F077
:10042A00013602360E2A9AEF01F001C002F0016A83
:10043A00000E0E8602644AEF02F0F00E0214D8A4EF
:10044A0029EF02F0023A0E84D89002BE9AEF01F028
:10045A0002360E2A02BE9AEF01F002360E2A02BEB8
:10046A009AEF01F002360E2A9AEF01F0010E0C6E95
:10047A00DFDE4DEF02F0020E0C6ED6DE4DEF02F01B
:10048A00040E0C6EE9DE4DEF02F0080E0C6EDDDE96
:02049A0012004E
:10049C000C6A0E6A0250D8A467EF02F001C002F099
:1004AC0000C001F0006A0E860250D8A467EF02F07B
:1004BC0001C002F0016A0E960E880250D8B479EF92
:1004CC0002F00E50035ED8A4D8A07EEF02F0D890B4
:1004DC0002BE83EF02F0003601360236032E6EEFB9
:1004EC0002F07EEF02F0010E0C6EAEDE86EF02F033
:1004FC00020E0C6E9CDE86EF02F0040E0C6E93DE88
:02050C001200DB
:10050E00A49EC1C875FF3EC4C2F83FC4C3F840C420
:10051E00C4F841C4C5F873A422D004013E513F1162
:10052E00401141111BE00801C251C311C411C51184
:10053E000EE1A5C6E1FFA6C6E2FF040EE66EA3C657
:10054E0000F0A4C601F099DE010E006E3BD0010E44
:10055E000801C25F000EC35BC45BC55BDCD73EC443
:10056E00C2F83FC4C3F840C4C4F841C4C5F8A4BE21
:10057E0022D004013E513F11401141111BE00801F0
:10058E00C251C311C411C5110EE1A5C6E1FFA6C625
:10059E00E2FF040EE66EA3C600F0A4C601F06DDE07
:1005AE00010E006E0FD0010E0801C25F000EC35B7C
:1005BE00C45BC55BDCD771BC02D0006A03D071840A
:0605CE00020E006E120097
:0E05D400550EA76EAA0EA76E0E01BF91120063
:1005E20003500718D8A405EF03F002500618D8A448
:1005F20005EF03F001500518D8A405EF03F00050F1
:0E0602000418D8B4D8841200D8941200120044
:0E061000550EA76EAA0EA76E0E01BF81120036
:10061E000801C151200A09E0C1510D0804E3090E79
:10062E00C15D01E302D0006A02D0010E006E12001D
:10063E003EC4C3F83FC4C4F840C4C5F841C4C6F8AC
:10064E000801C16BC26BC251120802E1C1518E0882
:10065E0008E31FDE005201E004D00801C14BC22B9B
:10066E00F2D70801120EC25D02E18F0EC15D03E3E7
:10067E007B0E006E26D0718071A022D004013E51F7
:10068E003F11401141111BE00801C351C411C511A6
:10069E00C6110EE1A5C6E1FFA6C6E2FF050EE66E87
:1006AE00A3C600F0A4C601F0E8DD010E006E09D06D
:1006BE00010E0801C35F000EC45BC55BC65BDCD7D1
:0406CE00006A1200AC
:1006D2000801C151390806E3300EC15D03E3010E82
:0806E200006E01D0006A120055
:1006EA000050086E0150006E0250016E0350026EF7
:1006FA00036A0B6A0C6A9E0E036E0A6A02AE92EFD6
:10070A0003F0081E001E011E021E082AD8B4002A81
:10071A00D8B4012AD8B4022A0A8E020E0C6EC8DD99
:02072A001200BB
:10072C00220E0C6E086A096A0A6A0B6A0C06D8B4A7
:10073C001FD0D8900B320A320932083203320232FF
:10074C0001320032D8A0F2D70C06D8B409D004502C
:10075C0008260550092206500A2207500B22EAD718
:10076C00045008260550092206500A2207500B2275
:02077C00120069
:08077E000B6A0B86FF0E12004E
:100786000B800BAECFEF03F0026A0AAEFF0E026ECD
:0C079600016E006E0A360232FF0E1200E7
:1007A200025006180E6E086A096A0B6A0350076443
:1007B200C4EF04F006500A6E068E028E03500B6ED2
:1007C2000750036E000E0B6414EF04F00B50075E2B
:1007D200D8B4B5EF04F0070E076483EF04F0075EA8
:1007E20000C008F001C000F002C001F0026A074E2A
:1007F200B5EF04F0076458EF04F0075E00C008F09C
:1008020001C000F0016A074EB5EF04F0076436EF4D
:1008120004F0075E00C008F0006A074EB5EF04F06E
:1008220007641DEF04F00AC002F005C001F004C025
:1008320000F0086AE1EF05F0030E076428EF04F008
:10084200075E08380F0B086E074EB5EF04F0D8901C
:100852000832074EB5EF04F0D8900832074EB5EFD4
:1008620004F0D8900832B5EF04F0030E076447EFA6
:1008720004F0075E08380F0B086E0038F00B0826EC
:1008820000380F0B006E074EB5EF04F0D89000321F
:100892000832074EB5EF04F0D89000320832074E06
:1008A200B5EF04F0D89000320832B5EF04F0030E31
:1008B20007646FEF04F0075E08380F0B086E00380C
:1008C200F00B082600380F0B006E0138F00B0026E3
:1008D20001380F0B016E074EB5EF04F0D8900132CC
:1008E20000320832074EB5EF04F0D89001320032E0
:1008F2000832074EB5EF04F0D890013200320832C8
:10090200B5EF04F0030E0764A0EF04F0075E0838A9
:100912000F0B086E0038F00B082600380F0B006E24
:100922000138F00B002601380F0B016E0238F00B74
:10093200012602380F0B026E074EB5EF04F0D89075
:100942000232013200320832074EB5EF04F0D8907D
:100952000232013200320832074EB5EF04F0D8906D
:100962000232013200320832096A000E0EAEA9EFDD
:1009720005F0081E001E011E021E082A0022012286
:100982000222A9EF05F00750D8A4CAEF04F0E1EF64
:1009920005F0096A02C00AF0028E068E0750035C57
:1009A200076ED8B49CEF05F0070E07646AEF05F0F6
:1009B200075E0450096E0550046E0650056E066A05
:1009C200074E9CEF05F0070E07643FEF05F0075E48
:1009D2000450096E0550046E056A074E9CEF05F03F
:1009E200070E07641DEF05F0075E0450096E046AE6
:1009F200074E9CEF05F0070E076404EF05F00AC0EE
:100A020002F0E1EF05F0030E07640FEF05F0075E59
:100A120009380F0B096E074E9CEF05F0D89009328A
:100A2200074E9CEF05F0D8900932074E9CEF05F077
:100A3200D89009329CEF05F0030E07642EEF05F003
:100A4200075E09380F0B096E0438F00B09260438CB
:100A52000F0B046E074E9CEF05F0D890043209325A
:100A6200074E9CEF05F0D89004320932074E9CEFF6
:100A720005F0D890043209329CEF05F0030E0764AA
:100A820056EF05F0075E09380F0B096E0438F00BBC
:100A9200092604380F0B046E0538F00B04260538BE
:100AA2000F0B056E074E9CEF05F0D890053204320D
:100AB2000932074E9CEF05F0D89005320432093214
:100AC200074E9CEF05F0D8900532043209329CEFB4
:100AD20005F0030E076487EF05F0075E09380F0B78
:100AE200096E0438F00B092604380F0B046E053822
:100AF200F00B042605380F0B056E0638F00B0526A1
:100B020006380F0B066E074E9CEF05F0D8900632A2
:100B1200053204320932074E9CEF05F0D8900632B6
:100B2200053204320932074E9CEF05F0D8900632A6
:100B3200053204320932086A000E0EAEA9EF05F042
:100B4200091E041E051E061E092A0422052206226B
:100B520009500826045000220550012206500222A4
:100B62000EBEC0EF05F0D8A0CFEF05F00232013281
:100B720000320832033ECFEF05F0DBEF05F0D8B0CC
:100B8200D5EF05F0000E081E001E011E021E082AE7
:100B92000022012202220A7ED5EF05F0010E0C6E20
:100BA2005DEC01F0E3EF05F0020E0C6E5DEC01F07E
:100BB200E3EF05F0040E0C6E31EC01F0E3EF05F00B
:060BC200000E0C6E120093
:100BC800C7B409D01F0EC514016E0150000A03E115
:0A0BD800010E006E01D0006A120049
:100BE2000A6A0350D8A40A800750D8A40A820A507D
:100BF200D8B454EF06F0030AD8B40DEF06F00AB0E9
:100C020008EF06F006AE52EF06F050EF06F002AE25
:100C120050EF06F052EF06F00250800B0A6E029E71
:100C22000650800B069E0A18D8B41EEF06F00A5032
:100C3200D8B450EF06F052EF06F00750035CD8B478
:100C420028EF06F0D8A044EF06F04AEF06F006506F
:100C5200025CD8B432EF06F0D8A044EF06F04AEFB7
:100C620006F00550015CD8B43CEF06F0D8A044EF82
:100C720006F04AEF06F00450005CD8B454EF06F0D8
:100C8200D8B04AEF06F00A52D8B452EF06F050EF4D
:100C920006F00A52D8B450EF06F052EF06F0D880B0
:0E0CA2001200D8901200D880D88412001200E0
:100CB000086A096A000E07620364DDEF06F002505D
:100CC00006180A6E075003267E0ED8A06EEF06F0B7
:100CD000035ED8B0E2EF06F072EF06F0035ED8A034
:100CE000E7EF06F0028E068E02C00EF001C00BF098
:100CF00000C00DF000500402F4CF0CF001500502CA
:100D0000F4CF00F0F3CF08F00402F3500C26F450B7
:100D10000822000E00220D500502F3500C26F4505C
:100D20000822000E002202500402F3500826F4505C
:100D3000002202500502016A000E0122F350002633
:100D4000F45001220D500602F3500826F450002200
:100D5000026A000E012202220B500602F350002606
:100D6000F4500122000E02220E500602F35001261A
:100D7000F450022202BEC5EF06F0083600360136F6
:100D800002360306D8B4E7EF06F0D8EF06F0D880B5
:100D9000800E08640030000E002201220222D8A03A
:100DA000D8EF06F0023201320032034AE2EF06F0D9
:100DB0000AAE029E000EEAEF06F0010E2AEC01F0E8
:100DC000EAEF06F0020E31EC01F0EAEF06F0040E55
:060DD0001DEC01F0120011
:040DD6007184120012
:100DDA0031DC780E0801C16F87EC02F050EC01F0AB
:100DEA000050000A01E1FAD7800E0801C16F87ECB2
:100DFA0002F050EC01F00050000A01E1FAD7B6C83F
:100E0A00C1F887EC02F050EC01F00050000A01E151
:100E1A00FAD7DCDF50EC01F00050000A01E1FAD702
:020E2A001200B4
:100E2C0008DC780E0801C16F87EC02F050EC01F081
:100E3C000050000A01E1FAD7400E0801C16F87EC9F
:100E4C0002F050EC01F00050000A01E1FAD7B6C8EC
:100E5C00C1F887EC02F0B2DE0050000A01E1FBD7CA
:040E6C00B4DF1200DD
:100E7000086A096A100E0C6E0134083609360450EF
:100E8000085E0550D8A0053C095ED8B007D00450D4
:100E900008260550D8B0053C0926D8900036013602
:060EA0000C2EEAD712003F
:100EA6000801B651180808E3B6510D0804E2110E00
:100EB600B65D01E201D002D0006AFAD1B751000A4C
:100EC600D8A48FD0B95302E0EAEC02F042D0B8C8F9
:100ED600C0FE82D0B8C8C1FE7FD0B8C8C2FE7CD0E2
:100EE600B8C8C3FE79D0B8C8C4FE76D0B8C8C5FEA7
:100EF60073D0B8C8C6FE70D0B8C8C7FE6DD0B8C823
:100F0600C8FE6AD0B8C8C9FE67D0B8C8CAFE64D0E1
:100F1600B8C8CBFE61D0B8C8CCFE5ED0B8C8CDFE8E
:100F26005BD0B8C8D1FE58D0B8C8D2FE55D0B8C824
:100F3600D3FE52D0B8C8D4FE4FD0B8C8D5FE4CD0D8
:100F4600B8C8D6FE49D0B8C8D7FE46D0B8C8D8FE6D
:100F560043D00801B651000ABAE0B651010ABAE018
:100F6600B651020ABAE0B651030ABAE0B651040A0B
:100F7600BAE0B651050ABAE0B651060ABAE0B65169
:100F8600070ABAE0B651080ABAE0B651090ABAE049
:100F9600B6510A0ABAE0B6510B0ABAE0B6510C0AC3
:100FA600BAE0B6510D0ABAE0B651110ABAE0B65126
:100FB600120ABAE0B651130ABAE0B651140ABAE0F8
:100FC600B651150ABAE0B651160ABAE0B651170A72
:100FD600BAE0B651180ABAE00801B95302E008ECC3
:100FE60003F00801B751010AD8A477D0B95302E03B
:100FF600EAEC02F036D0B6C8E1FE6AD0B6C8E2FE28
:1010060067D0B6C8E3FE64D0B6C8E4FE61D0B6C801
:10101600E6FE5ED0B6C8E7FE5BD0B6C8E8FE58D09E
:10102600B6C8E9FE55D0B6C8EAFE52D0B6C8F2FE3A
:101036004FD0B6C8F3FE4CD0B6C8F4FE49D0B6C8F9
:10104600F7FE46D0B6C8F8FE43D0B6C8FCFE40D080
:10105600B6C8FDFE3DD0B6C8FEFE3AD0B6C8FFFE05
:1010660037D00801B851000AC6E0B851010AC6E0F7
:10107600B851020AC6E0B851030AC6E0B851040ADC
:10108600C6E0B851050AC6E0B851060AC6E0B8512E
:10109600070AC6E0B851080AC6E0B851090AC6E010
:1010A600B8510A0AC6E0B8510B0AC6E0B8510C0A94
:1010B600C6E0B8510D0AC6E0B8510E0AC6E0B851EE
:1010C6000F0AC6E0B851100AC6E0B851110AC6E0C8
:1010D6000801B95302E008EC03F09AD00801B7B151
:1010E60002D0929001D09280E1D00801B7B102D02F
:1010F600929201D09282DAD00801B7B102D0929AC8
:1011060001D0928AD3D00801B7B102D0939001D012
:101116009380CCD00801B7B102D0939201D09382CC
:10112600C5D00801B7B102D0939401D09384BED044
:101136000801B7B102D0939601D09386B7D00801C3
:10114600B7B102D0939801D09388B0D00801B7B157
:1011560002D0939A01D0938AA9D00801B7B102D0E0
:10116600939C01D0938CA2D00801B7B102D0939E74
:1011760001D0938E9BD00801B7B102D0949001D0D4
:10118600948094D00801B7B102D0949201D0948291
:101196008DD00801B7B102D0949401D0948486D042
:1011A6000801B7B102D0949C01D0948C7FD008017D
:1011B600B7B102D0949E01D0948E78D00801B7B111
:1011C60002D0959401D0958471D00801B7B102D0B0
:1011D600959601D095866AD00801B7B102D0959848
:1011E60001D0958863D00801B7B102D0959A01D095
:1011F600958A5CD00801B7B102D0959C01D0958C38
:1012060055D00801B7B102D0959E01D0958E4ED02B
:101216000801B651000AD8B461D7B651010AD8B44C
:1012260064D7B651020AD8B467D7B651030AD8B400
:101236006AD7B651040AD8B46DD7B651050AD8B4E0
:1012460070D7B651060AD8B473D7B651070AD8B4C0
:1012560076D7B651080AD8B479D7B651090AD8B4A0
:101266007CD7B6510A0AD8B47FD7B6510B0A83E0A9
:10127600B6510C0A87E0B6510D0A8BE0B651110A39
:101286008FE0B651120A93E0B651130A97E0B651B1
:10129600140A9BE0B651150A9FE0B651160AA3E060
:1012A600B651170AA7E0B651180AABE0FF0E006E5A
:0212B600120024
:1012B8000B6A0A6A096A00500402F4CF09F0F3CFF6
:1012C80008F001500502F4CF0BF0F3CF0AF00050FC
:1012D8000502F3500926F4500A22E86A0B2201504D
:1012E8000402F3500926F4500A22E86A0B2208C0C7
:1012F80000F009C001F00AC002F00BC003F01200B0
:101308000B6A0350D8B4CAEF09F002500A6E028E75
:101318008E0E035E03AECEEF09F0036C080E035C7D
:10132800D8A0A9EF09F0036E013602C001F0026AE5
:10133800080E035CD8A0A9EF09F0036E0136016A14
:101348000350D8A4D890B3EF09F00350D8B4B3EF42
:1013580009F0D89002320132032EADEF09F00BBC30
:1013680001A0C0EF09F0D8A0C0EF09F0012AD8B455
:10137800022A02BEDDEF09F00AAEE3EF09F0021E11
:10138800011E012AD8B4022AE3EF09F0026A016AB1
:10139800E3EF09F00B800BAEE7EF09F0026A0AAE43
:1013A800E7EF09F0FF0E026E016E0A360232E7EF30
:1013B80009F0010E0C6EC3EC03F0E9EF09F0000E22
:1013C8000C6EE9EF09F0FF0E0C6E0150006E025032
:0413D800016E120090
:1013DC0000C008F00150006E016A026A036A0B6AD1
:1013EC000C6A016A026A036A960E036E0A6A00AE00
:1013FC0006EF0AF0081E001E082AD8B4002A0A8E2E
:10140C0000C001F008C000F0086A026A4EEC02F05D
:02141C001200BC
:10141E00086A080E0C6E003408360450085ED8B008
:0E142E0002D00826D89000360C2EF5D71200FA
:10143C000450000A12E10550000A0FE10650000AA0
:10144C000CE10750000A09E1FF0E006EFF0E016E61
:10145C007F0E026EFF0E036EA8D0086A096A075051
:10146C00D8B4C9EF0AF00350D8B4CEEF0AF002504A
:10147C0006180A6E028E068E0E6A02C008F001C0B3
:10148C000CF000C00DF004500D5E0550D8A0053CCA
:10149C000C5E0650D8A0063C085E086A0C6A0D6A01
:1014AC00D8A060EF0AF0D890023201320032083234
:1014BC00010E0E6E0750035ED8A06DEF0AF07E0E83
:1014CC000E240326D8B0D3EF0AF073EF0AF07E0E89
:1014DC000E240326D8A0D8EF0AF0180E0B6E0D368A
:1014EC000C3608360036013602360E360450005ED5
:1014FC000550D8A0053C015E0650D8A0063C025E03
:10150C0006340E120EA08EEF0AF00D8099EF0AF041
:10151C00045000260550D8B0053C01260650D8B022
:10152C00062802260D900B2E75EF0AF0BFEF0AF07D
:10153C00D8900036013602360E360450005E055047
:10154C00D8A0053C015E0650D8A0063C025E0634CD
:10155C000E10010B0D26D8B00C2AD8B4082AD8A42A
:10156C00BFEF0AF008320C320D32032AD8B4D3EF95
:10157C000AF00AAE089E0850026E0C50016E0D5017
:10158C00006EDBEF0AF0010EBFEC03F0DBEF0AF0AC
:10159C00020E2AEC01F0DBEF0AF0040E31EC01F044
:0C15AC00DBEF0AF0080E1DEC01F012004D
:0815B800067ED1EC03F01200E5
:1015C0000B6A0C6A086A0350D8B464EF0BF002C0CF
:1015D0000AF0028E9E0E035E03AE54EF0BF0036C16
:1015E000080E035CD8A021EF0BF0036E083600C094
:1015F00008F001C000F002C001F0026A080E035CAE
:10160000D8A021EF0BF0036E083600C008F001C02F
:1016100000F0016A080E035CD8A021EF0BF0036E06
:10162000083600C008F0006A080E035CD8A021EF5D
:101630000BF0036E0836086A0350D8A4D8902DEF3B
:101640000BF00350D8B42DEF0BF0D89002320132DA
:1016500000320832032E25EF0BF00BBC08A03EEF42
:101660000BF0D8A03EEF0BF0082AD8B4002AD8B46B
:10167000012AD8B4022A02BE68EF0BF00AAE64EF6A
:101680000BF0021E011E001E081E082AD8B4002AF4
:10169000D8B4012AD8B4022A64EF0BF0026A016AB6
:1016A000006A086A64EF0BF00B800BAE6FEF0BF073
:1016B000026A0AAE6FEF0BF0026E016E006E086EEA
:1016C0000A3602326FEF0BF00C6A000E70EF0BF06F
:1016D000010E0C6E000EC3EC03F070EF0BF0FF0E6A
:1016E0000250036E0150026E0050016E0850006EF1
:0216F0001200E6
:1016F2000801B851B91108E0B8C8E1FFB9C8E2FF62
:10170200B6C8E6FFB7C8E6FFB6C8E9FFB7C8EAFF42
:10171200EECF00F000C0BCF800C0C1F80FEC03F03F
:10172200005203E0B64BB72BEFD7BA6B000EBCBF2B
:10173200FF0E006E000E001802E12D0EBC1905E12D
:10174200010EBA6FB64BB72B0CD0000EBCBFFF0E0A
:10175200006E000E001802E12B0EBC1902E1B64B1E
:10176200B72BBC6BBD6BBE6BBF6BC06BBB6BBAB92F
:101772000BD0B6C8E9FFB7C8EAFFEE502E0A04E163
:10178200BA89B64BB72B59D0B6C8E9FFB7C8EAFF3A
:10179200EECFC1F869EC03F0005201E14FD0BA83F9
:1017A200000EBCBFFF0E000A02E1080EBC1940E0A9
:1017B200BAA901D0BB07BC2BBDC800F0BEC801F05E
:1017C200BFC802F0C0C803F00A0E046E000E056E18
:1017D200066E076E96EC03F000C0BDF801C0BEF8BD
:1017E20002C0BFF803C0C0F800000000B6C8E9FF9D
:1017F200B7C8EAFF300EEE5C006E016A000E015AB5
:10180200000E01BEFF0E026E036EBD510026BE51D8
:101812000122BF510222C051032200C0BDF801C003
:10182200BEF802C0BFF803C0C0F80000000003D039
:10183200BAB901D0BB2BB64BB72B99D7BC6BB6C884
:10184200E9FFB7C8EAFFEE50650A08E0B6C8E9FF4B
:10185200B7C8EAFFEE50450A01E068D0B64BB72B95
:10186200B6C8E9FFB7C8EAFFEE502D0A04E1BA870D
:10187200B64BB72B09D0B6C8E9FFB7C8EAFFEE509E
:101882002B0A02E1B64BB72BB6C8E9FFB7C8EAFF8D
:10189200EE50300A03E1B64BB72BF6D7B6C8E9FFD4
:1018A200B7C8EAFFEECFC1F869EC03F0005239E0A5
:1018B200B6C8E9FFB7C8EAFF300EEE5CBC6FB64BA4
:1018C200B72BB6C8E9FFB7C8EAFFEECFC1F869EC9B
:1018D20003F0005226E00A0EBC03F3CFBCF8B6C8F0
:1018E200E9FFB7C8EAFF300EEE5C006E0050BC277D
:1018F200B64BB72BB6C8E9FFB7C8EAFFEECFC1F8BF
:1019020069EC03F000520DE00A0EBC03F3CFBCF801
:10191200B6C8E9FFB7C8EAFF300EEE5C006E0050B1
:10192200BC27BAA703D0BC510008BC6FBC51BB276F
:10193200000EB91902E1000EB8190AE0BAA308D0E4
:10194200B8C8E1FFB9C8E2FFB6C8E6FFB7C8E6FF0C
:10195200BDC800F0BEC801F0BFC802F0C0C803F0A5
:1019620075EC03F000C0BDF801C0BEF802C0BFF8BC
:1019720003C0C0F8046A056A066A076ABDC800F0B7
:10198200BEC801F0BFC802F0C0C803F0F1EC02F01B
:10199200010ED8A4000E006E005205E0006A016A32
:1019A200026A036A04D1800EBB19006E800E000A1F
:1019B200005CD8B073D0BB510008BB6F800EBB195E
:1019C200006E800E0A0A005C1DE3BDC800F0BEC8AE
:1019D20001F0BFC802F0C0C803F0FF0E046EE60EAD
:1019E200056E5B0E066E5D0E076E58EC06F000C0CB
:1019F200BDF801C0BEF802C0BFF803C0C0F80A0EAD
:101A0200BB5FDCD7BB51000A1CE0BDC800F0BEC8FA
:101A120001F0BFC802F0C0C803F0CD0E046ECC0EB8
:101A2200056E4C0E066E7B0E076E58EC06F000C07B
:101A3200BDF801C0BEF802C0BFF803C0C0F8BB07C2
:101A4200E1D7010E046E000E056E000E066E010E49
:101A5200076EBDC800F0BEC801F0BFC802F0C0C822
:101A620003F0F1EC05F0010ED8B0000E006E00524A
:101A720014E0BAA109D0010E006E000E016E800EB4
:101A8200026E030E036E93D0010E006E000E016E05
:101A9200000E026E010E036E8AD072D0800E000A12
:101AA200006E800EBB19005C6BE20A0EBB5D1DE38B
:101AB200BDC800F0BEC801F0BFC802F0C0C803F044
:101AC200F90E046E020E056E150E066EA00E076E5E
:101AD20058EC06F000C0BDF801C0BEF802C0BFF865
:101AE20003C0C0F80A0EBB5FE0D7BB51000A1CE07E
:101AF200BDC800F0BEC801F0BFC802F0C0C803F004
:101B0200000E046E000E056E200E066E820E076E2B
:101B120058EC06F000C0BDF801C0BEF802C0BFF824
:101B220003C0C0F8BB07E1D7BDC804F0BEC805F0CA
:101B3200BFC806F0C0C807F0FF0E006EFF0E016EB0
:101B42007F0E026EFF0E036EF1EC05F0010ED8B0AF
:101B5200000E006E005214E0BAA109D0FF0E006E12
:101B6200FF0E016EFF0E026EFF0E036E20D0FF0EFF
:101B7200006EFF0E016E7F0E026EFF0E036E17D017
:101B8200BAA10DD0000EBD19006E000EBE19016E75
:101B9200800EBF19026E000EC019036E08D0BDC8B8
:101BA20000F0BEC801F0BFC802F0C0C803F01200C6
:101BB2000801A551000805E3070EA66F000EA76FE6
:101BC20012D0A551160805E2170EA86F000EA96FD4
:101BD20006D0A551010FA86FA96B000EA923A8C8B2
:101BE200A6F8A9C8A7F8A6C8B0F8A7C8B1F8AA6B02
:101BF200AB6B046A056A066A076A9FC800F0A0C850
:101C020001F0A1C802F0A2C803F0F1EC05F0010E48
:101C1200D8B0000E006E005209E0A3C8E1FFA4C8CC
:101C2200E2FF2D0EE66EA34BA42BA17F9FC804F00A
:101C3200A0C805F0A1C806F0A2C807F0006A016AB0
:101C4200026A036AF1EC05F0010ED8B0000E006ED4
:101C5200005237E0000E046E000E056E000E066E96
:101C62007F0E076E9FC800F0A0C801F0A1C802F065
:101C7200A2C803F0F1EC05F0010ED8B0000E006E20
:101C820000521FE09FC800F0A0C801F0A1C802F0F6
:101C9200A2C803F0000E046E000E056E200E066E42
:101CA200820E076E58EC06F000C09FF801C0A0F843
:101CB20002C0A1F803C0A2F8010EAA5F000EAB5B3E
:101CC200C9D7000E046E000E056E200E066E820E3F
:101CD200076E9FC800F0A0C801F0A1C802F0A2C818
:101CE20003F0F1EC05F0000ED8B0010E006E0052C8
:101CF2001EE0000E046E000E056E200E066E820EB1
:101D0200076E9FC800F0A0C801F0A1C802F0A2C8E7
:101D120003F01EEC0AF000C09FF801C0A0F802C058
:101D2200A1F803C0A2F80801AA4BAB2BCAD7AA514B
:101D3200B027AB51B123010EAC6F000EAD6F000E98
:101D4200B26F000EB36F000EB46F7F0EB56F800ED0
:101D5200AD19006E800EB119005C02E1B051AC5DAC
:101D62001EE2000E046E000E056E200E066E820E3E
:101D7200076EB2C800F0B3C801F0B4C802F0B5C82B
:101D820003F01EEC0AF000C0B2F801C0B3F802C0C2
:101D9200B4F803C0B5F80801AC4BAD2BD8D7000E90
:101DA200046E000E056E000E066E800E076EB2C83F
:101DB20000F0B3C801F0B4C802F0B5C803F01EECDD
:101DC2000AF09FC804F0A0C805F0A1C806F0A2C896
:101DD20007F0D1EC03F000C09FF801C0A0F802C0E8
:101DE200A1F803C0A2F8000E046E000E056E200ECC
:101DF200066E820E076EF1EC05F0000ED8B0010EF1
:101E0200006E00520BE0000E08019F6F000EA06FE3
:101E1200000EA16F7F0EA26FAA4BAB2B0801800EA2
:101E2200AB19006E800E005C02E1000EAA5D38E282
:101E3200A3C8E1FFA4C8E2FF300EE66EA34BA42BB9
:101E4200A3C8E1FFA4C8E2FF2E0EE66EA34BA42BAB
:101E5200800EB119006E800E005C02E1000EB05DD2
:101E620004E2B051AA5FB151AB5BFF0EAC6FFF0E43
:101E7200AD6F800EAB19006E800EAD19005C02E1F1
:101E8200AC51AA5D0DE2A3C8E1FFA4C8E2FF300E87
:101E9200E66EA34BA42B010EAC5F000EAD5BE9D73F
:101EA200AC6BAD6B800EAD19006E800EB119005C8B
:101EB20002E1B051AC5D63E29FC800F0A0C801F03E
:101EC200A1C802F0A2C803F084EC09F000C0AEF889
:101ED20001C0AFF8300E0026A3C8E1FFA4C8E2FF9C
:101EE20000C0E6FFA34BA42BAD51AB1902E1AA51EE
:101EF200AC1908E1A3C8E1FFA4C8E2FF2E0EE66E0A
:101F0200A34BA42BAEC800F0AFC801F0EEEC09F071
:101F120000C0B2F801C0B3F802C0B4F803C0B5F80B
:101F220000C004F001C005F002C006F003C007F0D3
:101F32009FC800F0A0C801F0A1C802F0A2C803F037
:101F4200DCEC0AF000C09FF801C0A0F802C0A1F8C2
:101F520003C0A2F8000E046E000E056E200E066E7F
:101F6200820E076E58EC06F000C09FF801C0A0F880
:101F720002C0A1F803C0A2F8AC4BAD2B93D7A3C803
:0A1F8200E1FFA4C8E2FFE66A1200C6
:101F8C009FC8F6FFA0C8F7FFA1C8F8FF0900F5CF5E
:101F9C0000F0005215E0ADB201D0FDD79FC8F6FF9E
:101FAC00A0C8F7FFA1C8F8FF0900F5CFC7F812ECDD
:101FBC0001F0010E08019F27000EA023A123E0D7FA
:021FCC00120001
:101FCE00840ED56E6D0ED76E840ED66E08014E93AE
:081FDE00D08EF294F28A120089
:101FE6009FC8B6F8A0C8B7F8A1C8B8F80801B96B79
:061FF60053EC07F012009D
:101FFC00A1C8F6FFA2C8F7FFA3C8F8FF0900F5CFE8
:10200C0000F0005218E0A1C8F6FFA2C8F7FFA3C861
:10201C00F8FF0900F5CF00F09FC8E1FFA0C8E2FF70
:10202C0000C0E6FF08019F4BA02B010EA127000E5C
:10203C00A223A323DDD79FC8E1FFA0C8E2FFE66A75
:02204C00120080
:10204E009FC804F0A0C805F004C002F005C003F05C
:10205E00044A052AA1C800F0A2C801F00801A14B4C
:10206E00A22B00C0E9FF01C0EAFF02C0E1FF03C0DE
:10207E00E2FFEECFE6FF02C0E9FF03C0EAFFEE5239
:0E208E0001E0E2D79FC800F0A0C801F01200E8
:10209C000D0E0801C76F12EC01F00A0E0801C76F94
:0620AC0012EC01F012002D
:1020B2009FC804F0A0C805F004C0E9FF05C0EAFF0C
:1020C200EE5203E0044A052AF7D704C002F005C025
:1020D20003F0044A052AA1C800F0A2C801F00801D1
:1020E200A14BA22B00C0E9FF01C0EAFF02C0E1FF41
:1020F20003C0E2FFEECFE6FF02C0E9FF03C0EAFF42
:10210200EE5201E0E2D79FC800F0A0C801F0120031
:102112009FC8E9FFA0C8EAFFEE500801A11905E136
:102122009FC800F0A0C801F010D09FC800F0A0C85E
:1021320001F09F4BA02B00C0E9FF01C0EAFFEECFE8
:0C21420000F00052E5E1006A016A1200A2
:10214E000801A26B9FC8E9FFA0C8EAFFEECFA1F875
:10215E00A151000A0FE0A1C8C7F812EC01F0080166
:10216E00A22BA2519F25E96E000EA021EA6EEECFA2
:06217E00A1F8EED71200EB
:10218400080E0C6EC10E0D6E0D2EFED70C2EFCD754
:0621940000000000120033
:10219A009FC8B6F8A0C8B7F80801B86BB96B79EC54
:0421AA000BF0120024
:1021AE009FC802F0A0C803F002C000F003C001F007
:1021BE00024A032A00C0E9FF01C0EAFFEE5201E025
:1021CE00F3D708019F51025C006EA0510358016EB7
:0A21DE00010E005E000E015A12000F
:1021E800200E0801B66FEDEC06F00801B66BEDECB9
:1021F80006F0210E0801B66FEDEC06F09FC8B6F8A0
:10220800EDEC06F008019F510F0FB66FEDEC06F0EC
:10221800220E0801B66FEDEC06F0010E0801B66F4C
:10222800EDEC06F0030E0801B66FEDEC06F00801C0
:10223800A16BA26B800EA219006E800E005C02E1F9
:10224800300EA15D24E2030E006E000E016EA0C8E0
:1022580004F0000E056E5CEC09F01D0E0024E96E1A
:10226800040E0120EA6EA151EE24F66EA251EE2072
:10227800F76E000EA2BFFF0EEE20F86E0900F5CF34
:10228800B6F816EC07F00801A14BA22BD3D7120021
:10229800A2C800F0016A026A036AFF0E0016000E67
:1022A800011600C0A7F801C0A8F87F0E005C026EF6
:1022B800000E0158036E02C0A7F803C0A8F8800EEC
:1022C8000318006E800E005C02E1000E025C22E240
:1022D800046A056A066A076A9FC800F0A0C801F088
:1022E800A1C802F0A2C803F0F1EC05F0010ED8B0C5
:1022F800000E006E005209E0000E006E000E016E26
:10230800800E026E7F0E036E5CD0006A016A026A5C
:10231800036A57D00801A851000802E1A75118081C
:1023280009E29FC800F0A0C801F0A1C802F0A2C845
:1023380003F047D09FC800F0A0C801F0A1C802F080
:10234800A2C803F0E0EC0AF075EC03F000C0A3F8B3
:1023580001C0A4F802C0A5F803C0A6F800C004F0A4
:1023680001C005F002C006F003C007F09FC800F0E6
:10237800A0C801F0A1C802F0A2C803F0F1EC05F072
:10238800010ED8B0000E006E005213E0000E046E6D
:10239800000E056E000E066E7F0E076EA3C800F0D5
:1023A800A4C801F0A5C802F0A6C803F0DCEC0AF046
:1023B80008D0A3C800F0A4C801F0A5C802F0A6C8B8
:0423C80003F012000C
:1023CC00020E0C6E350E0D6E0D2EFED70C2EFCD79C
:0623DC00000000001200E9
:0E23E200C70E0D6E0D2EFED70000000012007B
:1023F0009FC8F6FFA0C8F7FFA1C8F8FF0900F5CFF6
:1024000000F0005215E0A8B201D0FDD79FC8F6FF3A
:10241000A0C8F7FFA1C8F8FF0900F5CFC7F83DEC49
:1024200001F0010E08019F27000EA023A123E0D791
:02243000120098
:102432000801A16BA26B9FC803F0A0C804F09FC85B
:1024420005F0A0C806F003C0E9FF04C0EAFFEE50A1
:10245200200A04E1A151A21101E110D0010EA16FE5
:10246200000EA26F03C0E9FF04C0EAFF05C0E1FF4E
:1024720006C0E2FFEECFE6FF054A062A03C001F0DE
:1024820004C002F0034A042A01C0E9FF02C0EAFFC5
:10249200EE50000AD8E19FC800F0A0C801F0120077
:1024A2000801A36B050EA35D0AE2A351A125E16E0B
:1024B200000EA221E26E200EE66EA32BF3D7A351EB
:1024C200A125E16E000EA221E26EE66AA307A351E6
:1024D200A125A46F000EA221A56F0A0E046E000EA4
:1024E200056E9FC800F0A0C801F038EC07F008C0E4
:1024F20000F009C001F0300E0026A4C8E1FFA5C813
:10250200E2FF00C0E6FF0A0E046E000E056E9FC8D1
:1025120000F0A0C801F038EC07F000C09FF801C03D
:10252200A0F8000E011802E1000E001801E102D02D
:06253200A307CDD7120043
:0A253800000E9EBA010E006E1200A4
:10254200AFCF01F0ACA202D0AC98AC8801C000F0D1
:02255200120075
:10255400A3C800F00801A307005228E09FC8E9FFC0
:10256400A0C8EAFFEE50000A0CE09FC8E9FFA0C82B
:10257400EAFFA1C8D9FFA2C8DAFFEE50DE1801E1D4
:102584000FD09FC8E9FFA0C8EAFFA1C8D9FFA2C81D
:10259400DAFFDE50EE5C006E016A000E015A08D0CC
:1025A40008019F4BA02BA14BA22BD2D7006A016A32
:0225B400120013
:1025B6000D0E0801C76F3DEC01F00A0E0801C76F4A
:0625C6003DEC01F01200E3
:1025CC000801A051B00FB66FEDEC06F00F0E08012C
:1025DC009F15B66FEDEC06F0F00E08019F15B66F67
:1025EC00B633B69FB633B69FB633B69FB633B69FE7
:0825FC00B689EDEC06F01200B7
:102604000801A26B030EA25D0AE2A251A025E16EAD
:10261400000EA121E26E200EE66EA22BF3D7A2518A
:10262400A025E16E000EA121E26EE66AA207A25186
:10263400A025A36F000EA121A46F0A0E046E9FC8EB
:1026440000F00FEC0AF008C000F0300E0026A3C81A
:10265400E1FFA4C8E2FF00C0E6FF0A0E046E9FC8B3
:1026640000F00FEC0AF000C09FF80050000A01E1EE
:0826740002D0A207DCD712001E
:0E267C00030E0D6E0D2EFED7000000001200A2
:10268A000801A26B9FC8E9FFA0C8EAFFEECFA1F834
:10269A00A151000A0FE0A1C8C7F83DEC01F00801FA
:1026AA00A22BA2519F25E96E000EA021EA6EEECF61
:0626BA00A1F8EED71200AA
:1026C00093C801F0010E006E015004E00036009046
:1026D000FF0FFBD700C097F8001C0801966F956BA1
:1026E00091C8E9FF92C8EAFF946B9451070820E370
:1026F0009651EF16120EE9269651EF16BFDF97514D
:10270000EF12BCDF120EE95E9751EF14006E0CE081
:1027100094C801F0010E006E015004E000360090F4
:10272000FF0FFBD7005095135CDE5BDE942BDDD7EB
:0627300095C800F0120044
:1027360091C800F00032009E0032009E0032009EDA
:102746000032009E390E0024F66E630EF76E000E00
:10275600F722000EF86E000EF8220900F5CF00F001
:1027660092C8E1FF93C8E2FF00C0E6FF010E080130
:102776009225E16E000E9321E26E0F0E9115006E0A
:10278600390E0024F66E630EF76E000EF722000E69
:10279600F86E000EF8220900F5CF00F000C0E6FF43
:1027A600020E9225E16E000E9321E26EE66A120099
:1027B6007A0E0601A76F020EA86FC70EA96F080E44
:1027C600AA6FFF0E976FFF0E986F000E996F000E9F
:1027D6009A6FFF0E9B6FFF0E9C6F000E9D6F000E93
:1027E6009E6FFF0E9F6FFF0EA06F000EA16F000E73
:1027F600A26FA88A900E9C6EA4AA03D0AACF00F05E
:04280600FBD71200EA
:10280A0093C801F0010E006E015004E000360090FA
:10281A00FF0FFBD700C095F8001E91C8E9FF92C8C8
:10282A00EAFF0050EF16120EE9260050EF16A5DC5B
:10283A0008019551EF12120EE95EC3DD9551EF14AE
:10284A00946F9451000A000ED8A4010E946F95DC7F
:06285A0094C800F012001A
:1028600093C801F0010E006E015004E000360090A4
:10287000FF0FFBD700C097F8001E00C096F891C864
:10288000E9FF92C8EAFF0050EF16120EE926080190
:10289000956B9551070815E395C800F094C801F0B1
:1028A000005004E00132019EFF0FFBD79651EF1656
:1028B00001A002D09751EF1289DD9751EF12952BAD
:0C28C000E8D7120EE95E8DDD8CDD120001
:1028CC00040E0C6EE40E0D6E0D2EFED70C2EFCD7E6
:0428DC0000001200E6
:1028E0000900F5CFE6FF0006FBE10106F9E1120061
:1028F0000801916BEAEC02F0160E08019F6F010EC1
:10290000A06F0C0EA16FF3EC0FF00050FF0A02E174
:102910000801912B0801170E9F6FA06B060EA16F87
:10292000F3EC0FF00050FF0A02E10801912B08ECD4
:0829300003F091C800F0120051
:10293800240E0601A76F020EA86FC70EA96F080E16
:10294800AA6F420E976F250E986F000E996F000EB2
:102958009A6F380E9B6F250E9C6F000E9D6F000EB0
:102968009E6FFF0E9F6FFF0EA06F000EA16F000EEF
:10297800A26FAD8A900EAC6E948E949C9EAA03D0E2
:08298800AFCF00F0FBD71200F5
:10299000070E0B6E170E0C6E6A0E0D6E0D2EFED707
:0C29A0000C2EFCD70B2EFAD70000120002
:1029AC000401F46BF56B000EF55D02E1FF0EF45DB6
:1029BC0012E20E0EF425E16E050EF521E26EE66ACA
:1029CC00010EF425006E000EF521016E00C0F4F42A
:1029DC0001C0F5F4E8D7F46BF56B000EF55D02E180
:1029EC00600EF45D12E21C0EF425E16E060EF5216C
:1029FC00E26EE66A010EF425006E000EF521016E02
:102A0C0000C0F4F401C0F5F4E8D7F46BF56B000EDC
:102A1C00F55D02E1600EF45D12E2EC0EF425E16E60
:102A2C00070EF521E26EE66A010EF425006E000E2B
:102A3C00F521016E00C0F4F401C0F5F4E8D7DC0E0A
:102A4C0008019F6F060EA06F3A0EA16F640EA26F65
:102A5C00000EA36FFEEC0FF0740E08019F6F080EB2
:102A6C00A06F360EA16F640EA26F000EA36FFEEC6A
:102A7C000FF0FA0E08019F6F040EA06F320EA16FBB
:102A8C00640EA26F000EA36FFEEC0FF006017C6BC0
:102A9C007D6B0401F46BF56BA4AA02D0AACF7EF671
:102AAC0006017E6B0E6B0F6BA38A0401196B1A6BFC
:022ABC00120006
:102ABE0091C804F092C805F008019551961124E0D2
:102ACE00010E955F000E965B04C002F005C003F088
:102ADE00044A052A93C800F094C801F0934B942B36
:102AEE0000C0E9FF01C0EAFF02C0E1FF03C0E2FF40
:102AFE00EECFE6FF02C0E9FF03C0EAFFEECF00F023
:102B0E00005201E101D0D8D795C800F096C801F067
:102B1E00010E955F000E965B0050011008E004C098
:102B2E00E1FF05C0E2FFE66A044A052AEDD791C827
:082B3E0000F092C801F0120042
:102B460008019F6BA06B3FDD0801926B080E925D3A
:102B560028E29251B00FB66FEDEC06F0C70E0D6E7F
:102B66000D2EFED7000000000801B66BEDEC06F056
:102B7600100E0801B66FEDEC06F00801936B800E9F
:102B8600935D0DE291C8B6F816EC07F0C70E0D6E10
:102B96000D2EFED7000000000801932BF0D7922BD4
:042BA600D5D712006D
:102BAA000801886B896B000E895D02E1FF0E885D62
:102BBA0012E2EC0E8825E16E060E8921E26EE66AC3
:102BCA00010E8825006E000E8921016E00C088F86A
:102BDA0001C089F8E8D70601D56BD66B0801886B66
:102BEA00896B9EAA02D0AFCFD7F60601D76B080130
:082BFA004C6B4D6B9D8A12002B
:102C0200FF0E0F01486F1F0E496F948E949C846AC9
:102C12008D6A969C9284070ED26E41919586958418
:062C220092909292120054
:102C2800000E0801921902E1000E911936E091C8D0
:102C3800E9FF92C8EAFFEE5230E093C89FF894C8C3
:102C4800A0F8D7EC10F000C0A3F891C89FF892C87C
:102C5800A0F893C8A1F894C8A2F878DC000E01186F
:102C680002E1000E001805E191C800F092C801F0D9
:102C780016D0010E080191259F6F000E9221A06FBA
:102C880093C8E9FF94C8EAFFEECFA1F889EC10F0E9
:102C980000C091F801C092F8C3D7006A016A120017
:102CA80091C8E9FF92C8EAFFEECF93F8000E080139
:102CB800946F000E946F000E941902E1200E931980
:102CC80007E0000E941902E1090E931901E003D000
:102CD800914B922BE5D7956B966B976B986B000E83
:102CE800941902E12D0E931905E1974B982B914BFE
:102CF800922B08D0000E941902E12B0E931902E1D1
:102D0800914B922B91C8E9FF92C8EAFFEECF93F856
:102D1800000E946F000E946F93C8C1F869EC03F02D
:102D2800005219E095C800F096C801F00A0E046E2A
:102D3800000E056E5CEC09F0300E935D026E000E1D
:102D48009459036E02500024956F03500120966F2A
:102D5800914B922BD7D79751981108E095510008BD
:102D6800006E96C801F0000E015604D095C800F018
:062D780096C801F01200F4
:102D7E00AE0E0801B66FEDEC06F00D0E0B6E2D0EBD
:102D8E000C6ED70E0D6E0D2EFED70C2EFCD70B2E05
:102D9E00FAD700000000AF0E0801B66FEDEC06F09A
:102DAE00070E0B6E170E0C6E6A0E0D6E0D2EFED7E5
:102DBE000C2EFCD70B2EFAD70000B00E0801B66F02
:102DCE00EDEC06F00801B66BEDEC06F0070E08010F
:102DDE00B66FEDEC06F0200E0801B66FEDEC06F0C6
:102DEE00020E0801B66FEDEC06F0210E0801B66F6B
:102DFE00EDEC06F00801B66BEDEC06F07F0E080167
:102E0E00B66FEDEC06F0220E0801B66FEDEC06F093
:102E1E000801B66BEDEC06F0070E0801B66FEDEC8F
:102E2E0006F0A10E0801B66FEDEC06F0A40E080137
:102E3E00B66FEDEC06F0A60E0801B66FEDEC06F0DF
:102E4E00C80E0801B66FEDEC06F0D30E0801B66F92
:102E5E00EDEC06F0400E0801B66FEDEC06F0D50E67
:102E6E000801B66FEDEC06F0800E0801B66FEDECC2
:102E7E0006F0A80E0801B66FEDEC06F03F0E080145
:102E8E00B66FEDEC06F0D60E0801B66FEDEC06F05F
:102E9E00800E0801B66FEDEC06F0D90E0801B66F84
:102EAE00EDEC06F01F0E0801B66FEDEC06F0DA0E33
:102EBE000801B66FEDEC06F00801B66BEDEC06F00E
:102ECE00EE0E0801B66FEDEC06F0810E0801B66F3E
:102EDE00EDEC06F07F0E0801B66FEDEC06F02E0E4F
:102EEE000801B66FEDEC06F0DB0E0801B66FEDECE7
:102EFE0006F0400E0801B66FEDEC06F08D0E0801DF
:102F0E00B66FEDEC06F0140E0801B66FEDEC06F0A0
:0C2F1E00AF0E0801B66FEDEC06F01200DB
:102F2A000801936B946B010E976F000E986F1C0E3D
:102F3A009F6F060EA06FD7EC10F000C095F801C085
:102F4A0096F8070E916F000E926F800E9219006E1E
:102F5A00800E9619005C02E19551915DD8B0B8D106
:102F6A006FD11C0E9125E96E060E9221EA6EEECF04
:102F7A0001F001502C0A0EE1100E9325E16E060EA7
:102F8A009421E26EE66A936B946B020E976F000EC1
:102F9A00986F9BD1100E9325E16E060E9421E26E76
:102FAA001C0E9125E96E060E9221EA6EEECF00F014
:102FBA0000C0E6FF934B942B88D11C0E9125E96E35
:102FCA00060E9221EA6EEECF01F001502C0A0EE1B4
:102FDA00740E9325E16E080E9421E26EE66A936BF5
:102FEA00946B030E976F000E986F6FD1740E932532
:102FFA00E16E080E9421E26E1C0E9125E96E060E12
:10300A009221EA6EEECF00F000C0E6FF934B942BBC
:10301A005CD11C0E9125E96E060E9221EA6EEECF66
:10302A0001F001502C0A07E1936B946B040E976F21
:10303A00000E986F4AD11C0E9125E96E060E922158
:10304A00EA6EEECF00F000C090F8934B942B3DD17E
:10305A001C0E9125E96E060E9221EA6EEECF01F062
:10306A0001502C0A0EE1DC0E9325E16E060E942126
:10307A00E26EE66A936B946B050E976F000E986F7B
:10308A0024D1DC0E9325E16E060E9421E26E1C0E0D
:10309A009125E96E060E9221EA6EEECF00F000C08D
:1030AA00E6FF934B942B11D11C0E9125E96E060E67
:1030BA009221EA6EEECF01F001502C0A07E1936BE0
:1030CA00946B060E976F000E986FFFD01C0E912519
:1030DA00E96E060E9221EA6EEECF00F000C073F898
:1030EA00934B942BF2D01C0E9125E96E060E922179
:1030FA00EA6EEECF01F001502C0A07E1936B946B54
:10310A00070E976F000E986FE0D01C0E9125E96E9E
:10311A00060E9221EA6EEECF00F000C0F3F4934B54
:10312A00942BD3D01C0E9125E96E060E9221EA6EDD
:10313A00EECF01F001502C0A0EE10A0E9325E16E42
:10314A00050E9421E26EE66A936B946B080E976FF4
:10315A00000E986FBAD00A0E9325E16E050E9421DF
:10316A00E26E1C0E9125E96E060E9221EA6EEECFF2
:10317A0000F000C0E6FF934B942BA7D01C0E9125BC
:10318A00E96E060E9221EA6EEECF01F001502C0A8A
:10319A000EE1EB0E9325E16E040E9421E26EE66ACF
:1031AA00936B946B090E976F000E986F8ED0EB0E8F
:1031BA009325E16E040E9421E26E1C0E9125E96EB0
:1031CA00060E9221EA6EEECF00F000C0E6FF934BA6
:1031DA00942B7BD01C0E9125E96E060E9221EA6E85
:1031EA00EECF01F001502C0A0EE1FA0E9325E16EA2
:1031FA00040E9421E26EE66A936B946B0A0E976F43
:10320A00000E986F62D0FA0E9325E16E040E942197
:10321A00E26E1C0E9125E96E060E9221EA6EEECF41
:10322A0000F000C0E6FF934B942B4FD095C891F85D
:10323A0096C892F84AD095C891F896C892F845D09F
:10324A00000E981902E1010E9719D8B48AD6000E19
:10325A00981902E1020E9719D8B4AFD6000E981940
:10326A0002E1030E9719D8B4D4D6000E981902E1D8
:10327A00040E9719D8B4ECD6000E981902E1050E7F
:10328A009719D8B411D7000E981902E1060E9719AA
:10329A00D8B429D7000E981902E1070E9719D8B4A5
:1032AA0041D7000E981902E1080E9719D8B466D7CB
:1032BA00000E981902E1090E97198CE0000E981970
:1032CA0002E10A0E9719B2E0B6D7914B922B3DD67E
:0A32DA0097C800F098C801F0120038
:1032E40008014EA508D0D40E9F6F630EA06F000E88
:1032F400A16FC6EC0FF0DC0E08019F6F060EA06FE5
:10330400CDEC10F000C0D8F601C0D9F602C0DAF650
:1033140003C0DBF6000E046E000E056E480E066E4A
:10332400850E076E1EEC0AF000C04FF801C050F87D
:1033340002C051F803C052F800C09FF801C0A0F8C1
:1033440002C0A1F803C0A2F84CEC11F000C091F83F
:1033540001C092F802C093F803C094F891C84FF8E2
:1033640092C850F893C851F894C852F8000E046EED
:10337400000E056E480E066E850E076ED8C600F068
:10338400D9C601F0DAC602F0DBC603F01EEC0AF07F
:1033940091C804F092C805F093C806F094C807F0E9
:1033A400DCEC0AF000C08AF801C08BF802C08CF88B
:1033B40003C08DF8000E046E000E056E480E066EF6
:1033C400850E076E58EC06F0000E046E000E056EB6
:1033D400700E066E840E076E1EEC0AF091C804F09F
:1033E40092C805F093C806F094C807F0D1EC03F036
:1033F40000C0D8F601C0D9F602C0DAF603C0DBF685
:1034040008019051530A1AE1D8C600F0D9C601F058
:10341400DAC602F0DBC603F0000E046E000E056E81
:10342400800E066E7F0E076E58EC06F000C0D8F6CC
:1034340001C0D9F602C0DAF603C0DBF6D8C69FF89D
:10344400D9C6A0F8DAC6A1F8DBC6A2F8EC0EA36FC1
:10345400070EA46F060EA56FD9EC0DF0DC0E9F6F5E
:10346400060EA06FEC0EA16F070EA26F27EC10F0F2
:103474008E6B8F6B000E8F5D02E11F0E8E5D0BE273
:10348400530E8E25E16E080E8F21E26E200EE66E3D
:103494008E4B8F2BEFD7536B530E9F6F080EA06F7D
:1034A400EC0EA16F070EA26F27EC10F0530E9F6F66
:1034B400080EA06F580EA16F040EA26F59EC10F005
:1034C4004EA517D0EC0E9F6F070EA06FA7EC10F05F
:1034D400200EC76F12EC01F090C8C7F812EC01F08F
:1034E400CB0E08019F6F630EA06F000EA16FC6EC98
:1034F4000FF0740E08019F6F080EA06FCDEC10F052
:1035040000C084F801C085F802C086F803C087F8BB
:10351400000E046E000E056E480E066E850E076ED4
:103524001EEC0AF000C04FF801C050F802C051F878
:1035340003C052F800C09FF801C0A0F802C0A1F86F
:1035440003C0A2F84CEC11F000C091F801C092F84D
:1035540002C093F803C094F891C84FF892C850F889
:1035640093C851F894C852F8000E046E000E056E0C
:10357400480E066E850E076E84C800F085C801F0FB
:1035840086C802F087C803F01EEC0AF091C804F064
:1035940092C805F093C806F094C807F0DCEC0AF072
:1035A40000C08AF801C08BF802C08CF803C08DF803
:1035B400000E046E000E056E480E066E850E076E34
:1035C40058EC06F0000E046E000E056E700E066ECA
:1035D400840E076E1EEC0AF091C804F092C805F040
:1035E40093C806F094C807F0D1EC03F000C084F847
:1035F40001C085F802C086F803C087F8080173513A
:10360400570A1AE184C800F085C801F086C802F0A0
:1036140087C803F0000E046E000E056E800E066E61
:103624007F0E076E58EC06F000C084F801C085F8E0
:1036340002C086F803C087F884C89FF885C8A0F83C
:1036440086C8A1F887C8A2F8EC0EA36F070EA46F72
:10365400060EA56FD9EC0DF0740E9F6F080EA06FC7
:10366400EC0EA16F070EA26F27EC10F0530E9F6FA4
:10367400080EA06FEC0EA16F070EA26F59EC10F0AC
:10368400530E9F6F080EA06F5A0EA16F040EA26F07
:1036940059EC10F04EA517D0EC0E9F6F070EA06FDB
:1036A400A7EC10F0200EC76F12EC01F073C8C7F836
:1036B40012EC01F0800E08019F6F630EA06F000EE4
:1036C400A16FC6EC0FF0FA0E08019F6F040EA06FF5
:1036D400CDEC10F000C0F6F401C0F7F402C0F8F429
:1036E40003C0F9F400C09FF801C0A0F802C0A1F81B
:1036F40003C0A2F8EC0EA36F070EA46F010EA56F12
:10370400D9EC0DF0FA0E9F6F040EA06FEC0EA16FB2
:10371400070EA26F27EC10F0530E9F6F080EA06FD8
:10372400EC0EA16F070EA26F59EC10F04EA506D057
:10373400EC0E9F6F070EA06FA7EC10F0200E6B6FBE
:103744006C6B726B4EA52CD0980E9F6F630EA06F9E
:10375400000EA16FC6EC0FF00A0E08019F6F050E54
:10376400A06FA7EC10F08C0E9F6F630EA06F000E7D
:10377400A16FC6EC0FF0EB0E08019F6F040EA06F53
:10378400A7EC10F0AE0E9F6F630EA06F000EA16F3A
:10379400C6EC0FF0F3C4C7F812EC01F04EEC10F0D5
:1037A40008014EB511D0120E9F6F640EA06F000E6B
:1037B400A16FC6EC0FF0530E08019F6F080EA06FA7
:0A37C400A7EC10F04EEC10F012001C
:1037CE00200E0801B66FEDEC06F00801B66BEDECBD
:1037DE0006F0210E0801B66FEDEC06F091C8B6F8B2
:1037EE00EDEC06F008019151070FB66FEDEC06F007
:1037FE00220E0801B66FEDEC06F092C8B6F8EDECAD
:10380E0006F008019251010FB66FEDEC06F00801BB
:10381E00946B956B800E9519006E800E005C02E124
:10382E00070E945D24E2030E006E000E016E93C827
:10383E0004F0000E056E5CEC09F0420E0024E96EF9
:10384E00040E0120EA6E9451EE24F66E9551EE2090
:10385E00F76E000E95BFFF0EEE20F86E0900F5CF45
:10386E00B6F816EC07F00801944B952BD3D712003F
:10387E00010E08019B6F190E9F6F630EA06F000E55
:10388E00A16FF8EC11F091C89FF8920E0801A06F8D
:10389E00080EA16F02EC13F0920E9F6F080EA06F30
:1038AE0045EC13F0EC0E9F6F630EA06F000EA16F30
:1038BE00F8EC11F0C20E08019F6F630EA06F000EA0
:1038CE00A16FF8EC11F01FEC03F091C8C1F887EC72
:1038DE0002F000C09BF80050000A0CE0580E0801E0
:1038EE009F6F630EA06F000EA16FF8EC11F0080130
:1038FE009B6B0CD00801B80E9F6F630EA06F000E6D
:10390E00A16FF8EC11F0010E08019B6FEBEC06F0C5
:0A391E00DBEC12F09BC800F0120071
:103928000801966B92AF0BD0010E966F2D0E070112
:10393800EC6F0801911F921F914B922B04D0966B4C
:10394800200E0701EC6F91C800F092C801F0013217
:103958000032019E01320032019E01320032019E86
:1039680001320032019E00C093F80A0E046E0FEC7B
:103978000AF00A0E046E0FEC0AF008C000F0300ED0
:103988000024016E01C0EDF70150300A03E1070180
:10399800200EED6F07010A0E046E93C800F00FECBD
:1039A8000AF008C000F0300E0024EE6F91C894F8B9
:1039B80092C895F80F0E08019115006E92C801F093
:1039C800000E011600C094F801C095F8710E046E3F
:1039D800020E056E5CEC09F000C097F801C098F87B
:1039E80097C894F898C895F82E0E0701EF6FE80E5F
:1039F800046E030E056E97C800F098C801F038EC05
:103A080007F0300E0024F06F640E046E000E056E91
:103A180097C800F098C801F038EC07F00A0E046E59
:103A2800000E056E38EC07F008C000F009C001F080
:103A3800300E0024F16FF26BF36BF46BED0E08019E
:103A48009F6F070EA06F19EC12F09651010A17E14B
:103A580093C800F0000E016EE80E046E030E056EAA
:103A68005CEC09F0945100240401546F080195514D
:103A780001200401556F000E566F576F1AD093C876
:103A880000F0000E016EE80E046E030E056E5CEC8D
:103A980009F00801945100269551012200500008B0
:103AA8000401546F01C055F4000E5557000E566FAF
:083AB800576F96C800F01200E0
:103AC000A00E06018B6F020E8C6F000E8D6F000E24
:103AD0008E6F3E0E8F6F060E906F000E916F000E70
:103AE000926FFF0E7F6FFF0E806F000E816F000ED2
:103AF000826FFF0E836FFF0E846FFF0E856FFF0EC8
:103B0000866F0E0E876F050E886FC10E896F080EC7
:103B10008A6FD60E936F0D0E946F000E956F000E88
:103B2000966F959295908C928C9095829580739ECD
:083B3000739C380E726E120046
:103B38008D0E0801B66FEDEC06F0140E0801B66F95
:103B4800EDEC06F0AF0E0801B66FEDEC06F01200D2
:103B58003D0E0B6EE10E0C6E3F0E0D6E0D2EFED758
:0E3B68000C2EFCD70B2EFAD700000000120026
:103B7600A1EC12F091C852F492C853F4E7EC0FF09E
:103B86005B0E9F6F600EA06F000EA16FF8EC11F038
:103B960091C89FF892C8A0F8930E0801A16F080E6D
:103BA600A26F51EC12F0930E9F6F080EA06F45ECBA
:103BB60013F0660E9F6F630EA06F000EA16FF8ECF8
:103BC60011F09CEC12F00050000A04E108014EB31B
:0A3BD60001D0F7D7A1EC12F01200A5
:103BE000210E0801B66FEDEC06F00801B66BEDECA6
:103BF00006F07F0E0801B66FEDEC06F0220E08010C
:103C0000B66FEDEC06F00801B66BEDEC06F0070EB2
:103C10000801B66FEDEC06F0D30E0801B66FEDECBF
:103C200006F0400E0801B66FEDEC06F008019F6B40
:103C3000A06BE6EC12F00801916B080E915D28E292
:103C40009151B00FB66FEDEC06F0010E0801B66FA2
:103C5000EDEC06F0100E0801B66FEDEC06F0270E45
:103C60000D6E0D2EFED7000000000801926B800E35
:103C7000925D0CE2B66B16EC07F04F0E0D6E0D2E3A
:103C8000FED7000000000801922BF1D7912BD5D769
:103C90002E0EB66FEDEC06F008019F6BA06BE6EC04
:043CA00012F012000C
:103CA40008019A6B9B6B9C6B9D6B9E6B91C89DF8F6
:103CB40092C89EF891C89FF892C8A0F8E6EC12F05A
:103CC40038D108019C519325E96E000E9421EA6EC7
:103CD400EE50000A46E0050E9E5D43E29C5193259A
:103CE400E96E000E9421EA6E200EEE5C9A6F9D51EF
:103CF400780809E291C89DF89E2B91C89FF89EC848
:103D0400A0F8E6EC12F008019B6B060E9B5D25E221
:103D1400060E006E000E016E026E036E9AC804F069
:103D2400000E056E066E076E96EC03F0570E002625
:103D3400590E0122000E02229B510024F66E000E41
:103D44000120F76E000E0220F86E0900F5CFB6F8D8
:103D540016EC07F008019B2BD8D7060E9D279C2B49
:103D6400B0D7F4D093C89FF894C8A0F8D7EC10F05B
:103D740000C096F801C097F89C6B9C519325E96E9E
:103D8400000E9421EA6EEE50000AD8B475D00F0EDE
:103D94009C5D72E29C519325E96E000E9421EA6EBB
:103DA400200EEE5C9A6F9DC89FF89EC8A0F8E6ECC2
:103DB40012F008019B6B080E9B5D25E2040E026E57
:103DC4009AC800F0000E016E025005E00036009023
:103DD4000136FF0FFAD79B510026000E0122240E54
:103DE4000024F66E4F0E0120F76E000EF86E000EE2
:103DF40001BEFF0EF8220900F5CFB6F816EC07F065
:103E040008019B2BD8D79DC89FF89E51010FA06F26
:103E1400E6EC12F008019B6B080E9B5D29E2040E90
:103E2400026E9AC800F0000E016E025005E00036E2
:103E340000900136FF0FFAD79B510026000E012295
:103E4400080E0026000E0122240E0024F66E4F0EEA
:103E54000120F76E000EF86E000E01BEFF0EF82270
:103E64000900F5CFB6F816EC07F008019B2BD4D760
:103E7400080E9D279C2B81D769D093C89FF894C8BE
:103E8400A0F8D7EC10F000C098F801C099F8800EA3
:103E9400026E800E0118025C02E10050000847E245
:103EA4009B6B800E006E800E9919005C02E19851A4
:103EB4009B5D3DE2070E9B25966F976B000E972343
:103EC4009851965F9951975B040E006E005005E07F
:103ED400963796919737FF0FFAD79B519325E96E42
:103EE400000E9421EA6EEECF01F001C09AF8015061
:103EF4002F080BE23A0E9A5D08E296C89FF8300E3E
:103F04009A5DA06FF4EC10F010D09A512E0A07E1DC
:103F140096C89FF80A0EA06FF4EC10F006D096C86D
:103F24009FF8200EA06FF4EC10F09B2BBAD70ED0A4
:103F34000DD008019551010AD8B4C3D69551020A8F
:0E3F4400D8B410D79551030A98E0F2D71200B6
:103F52001FEC32F001EC16F008014E95899089921F
:103F6200190E04015C6F000E5D6F6B0E696F040E1B
:103F72006A6F89807E86270E7F6E0F0EB06EAD84CB
:103F82009CEC14F078EC14F000C05EF40050020ACD
:103F920003E108014E8D02D008014E9D7C86040E7D
:103FA2007D6EE10EAB6EA884DBEC13F0DBEC12F05D
:103FB200E90E08019F6F5B0EA06F000EA16FF8EC77
:103FC20011F0960E08019F6F5D0EA06F000EA16F9B
:103FD200F8EC11F0390E08019F6F5C0EA06F000E15
:103FE200A16FF8EC11F0860E08019F6F5C0EA06FB6
:103FF200000EA16FF8EC11F07F0E08019F6F5B0EAF
:10400200A06F000EA16FF8EC11F09E0E08019F6FD9
:10401200610EA06F000EA16FF8EC11F0FD0E080109
:104022009F6F600EA06F000EA16FF8EC11F0E20E10
:1040320008019F6F5F0EA06F000EA16FF8EC11F0E8
:10404200590E08019F6F5D0EA06F000EA16FF8EC74
:1040520011F0190E08019F6F5D0EA06F000EA16F87
:10406200F8EC11F00E0E08019F6F600EA06F000EAB
:10407200A16FF8EC11F0370E08019F6F610EA06F6F
:10408200000EA16FF8EC11F01A0E08019F6F610E7D
:10409200A06F000EA16FF8EC11F0C00E08019F6F27
:1040A200600EA06F000EA16FF8EC11F0DBEC12F0C5
:1040B200A39A9D9AF28C0D0E0B6E2D0E0C6ED70EDE
:1040C2000D6E0D2EFED70C2EFCD70B2EFAD700004C
:1040D20000000C0E0801C76F3DEC01F01F0E0B6EC5
:1040E200710E0C6E1E0E0D6E0D2EFED70C2EFCD711
:1040F2000B2EFAD700008982380E08019F6F600EDE
:10410200A06F000EA16FF8EC11F0C8EC14F00401DE
:104112005F6B606B800E0801916F0F0E926F020E43
:10412200936F05EC14F066EC14F0800E916F0F0E95
:10413200926F020E936F330E946F30EC14F066ECB4
:1041420014F0800E916F0F0E926F020E936F60EC5F
:1041520013F000C0D7F666EC14F0290E9F6F630EC1
:10416200A06F000EA16FF8EC11F00701EC6BD7C63F
:1041720091F8EC0E0801926F070E936F9BEC13F00F
:10418200EC0E9F6F070EA06FA7EC10F0FC0E9F6F56
:10419200630EA06F000EA16FC6EC0FF008018E6BCC
:1041A2008F6B000E8F5D02E1060E8E5D28E2800E9F
:1041B200916F0F0E926F020E936F60EC13F000C0BE
:1041C200D7F666EC14F0610E8E25E16E040E8F2197
:1041D200E26ED7C6E6FF0701EC6BD7C691F8EC0E8C
:1041E2000801926F070E936F9BEC13F0EC0E9F6F1A
:1041F200070EA06F45EC13F08E4B8F2BD2D7F40E27
:104202009F6F630EA06F000EA16FF8EC11F0800E8D
:104212000801916F0F0E926F020E936F60EC13F014
:1042220000C0D7F60701EC6BD7C691F8EC0E080177
:10423200926F070E936F9BEC13F0EC0E9F6F070EBD
:10424200A06F45EC13F0DBEC12F0070E08019F6F34
:10425200630EA06F000EA16FF8EC11F0800E080142
:10426200916F0F0E926F020E936F05EC14F0800E99
:10427200916F0F0E926F020E936FCC0E946F30EC13
:1042820014F0800E916F0F0E926F020E936F440E18
:10429200946F30EC14F066EC14F0800E916F0F0EF8
:1042A200926F020E936F05EC14F0800E916F0F0E59
:1042B200926F020E936FCC0E946F30EC14F0800E5E
:1042C200916F0F0E926F020E936FBE0E946F30ECD1
:1042D20014F0250E0B6E870E0C6E8B0E0D6E0D2ECE
:1042E200FED70C2EFCD70B2EFAD700000000800E52
:1042F200916F0F0E926F020E936F60EC13F000C07D
:104302001BF4000E04011C6F800E0801916F0F0E4A
:10431200926F020E936F60EC13F000C003F0026A1A
:1043220004011B510224006E1C510320016E00C0C7
:104332004EF401C04FF400C091F801C092F894EC21
:104342001CF0EC0E08019F6F070EA06F19EC12F023
:10435200EC0E9F6F070EA06FD7EC10F000C0AFF607
:1043620001C0B0F6EC0E00249F6F070E0120A06F73
:104372002D0EA16F640EA26F000EA36FFEEC0FF064
:10438200EC0E08019F6F070EA06F45EC13F0DBECFB
:1043920012F0DBEC12F0230E08019F6F620EA06F89
:1043A200000EA16FF8EC11F0780E746E60EC1DF047
:1043B20050EC01F00050000A01E1FAD7070E0B6E33
:1043C200170E0C6E6A0E0D6E0D2EFED70C2EFCD73C
:1043D2000B2EFAD70000780E0601B16F780E080195
:1043E200916F3FEC1CF000C0AFF6000E0601B06FFB
:1043F200740E08018E6F000E8F6F000E8F5D02E14A
:10440200820E8E5D25E28EC891F83FEC1CF000C052
:10441200AFF6000E0601B06F070E0B6E170E0C6E94
:104422006A0E0D6E0D2EFED70C2EFCD70B2EFAD770
:104432000000000E006EB051005C02E1AF510008B6
:1044420001E206D0020E08018E27000E8F23D5D777
:10445200070E0B6E170E0C6E6A0E0D6E0D2EFED72A
:104462000C2EFCD70B2EFAD70000000E0601B01955
:1044720002E1000EAF190DE1860E08019F6F610E79
:10448200A06F000EA16FF8EC11F08982899091EF74
:1044920027F0490E08019F6F630EA06F000EA16FF7
:1044A200C6EC0FF0730E08019F6F630EA06F000E33
:1044B200A16FF8EC11F0BFEC16F0070E0B6E170EA1
:1044C2000C6E6A0E0D6E0D2EFED70C2EFCD70B2E27
:1044D200FAD70000A30E08019F6F630EA06F000EB3
:1044E200A16FF8EC11F09CEC1DF0070E0B6E170E8D
:1044F2000C6E6A0E0D6E0D2EFED70C2EFCD70B2EF7
:10450200FAD70000FE0E0601AB6FFF0EAC6F6B0E0A
:104512000401696F040E6A6FF28EF0EC1DF069C43B
:104522009FF86AC4A0F8CB0E0801A16F610EA26FBA
:10453200000EA36FFEEC0FF00801916B926B69C441
:1045420093F86AC494F8010E956F52EC1EF069C498
:104552009FF86AC4A0F845EC13F0DBEC12F0ACEC67
:104562001DF0ACEC1DF0ACEC1DF069C49FF86AC400
:10457200A0F8B70E0801A16F620EA26F000EA36F22
:10458200FEEC0FF069C49FF86AC4A0F845EC13F082
:10459200DBEC12F0010E0801916F010E926F69C4FB
:1045A20093F86AC494F8010E956F52EC1EF0140E43
:1045B200916F000E926FBBEC1DF0F0EC1DF069C420
:1045C2009FF86AC4A0F8B50E0801A16F610EA26F30
:1045D200000EA36FFEEC0FF069C49FF86AC4A0F846
:1045E20045EC13F0DBEC12F00801916B926B69C49D
:1045F20093F86AC494F8010E956F52EC1EF069C4E8
:104602009FF86AC4A0F8D10EA16F5C0EA26F000ED3
:10461200A36FFEEC0FF0010E0801916F010E926F75
:1046220069C493F86AC494F8010E956F52EC1EF0B7
:10463200140E916F000E926FBBEC1DF0F0EC1DF0AA
:1046420069C49FF86AC4A0F8E10E0801A16F620E66
:10465200A26F000EA36FFEEC0FF069C49FF86AC44C
:10466200A0F845EC13F0DBEC12F00801916B926BB1
:1046720069C493F86AC494F8010E956F52EC1EF067
:1046820069C49FF86AC4A0F8CC0EA16F620EA26F33
:10469200000EA36FFEEC0FF0010E0801916F030EE6
:1046A200926F69C493F86AC494F8010E956F52EC44
:1046B2001EF0140E916F000E926FBBEC1DF0F0EC29
:1046C2001DF069C49FF86AC4A0F8A20E0801A16F88
:1046D200620EA26F000EA36FFEEC0FF069C49FF88A
:1046E2006AC4A0F845EC13F0DBEC12F00801916B00
:1046F200926B69C493F86AC494F8010E956F52ECF8
:104702001EF069C49FF86AC4A0F84E0EA16F620E33
:10471200A26F000EA36FFEEC0FF0010E0801916F65
:10472200010E926F69C493F86AC494F8020E956FF1
:1047320052EC1EF0140E916F000E926FBBEC1DF046
:10474200F0EC1DF0040E0B6E0C0E0C6E330E0D6EA3
:104752000D2EFED70C2EFCD70B2EFAD70000000030
:1047620069C49FF86AC4A0F8390E0801A16F620EED
:10477200A26F000EA36FFEEC0FF069C49FF86AC42B
:10478200A0F845EC13F0916B926B69C493F86AC47C
:1047920094F8010E956F52EC1EF069C49FF86AC43A
:1047A200A0F8200EA16F640EA26F000EA36FFEECA4
:1047B2000FF069C49FF86AC4A0F845EC13F0DBEC73
:1047C20012F0010E0801916F010E926F69C493F805
:1047D2006AC494F8030E956F52EC1EF0140E916F9A
:1047E200000E926FBBEC1DF0F0EC1DF0040E0B6E90
:1047F2000C0E0C6E330E0D6E0D2EFED70C2EFCD74A
:104802000B2EFAD70000000069C49FF86AC4A0F812
:104812006D0E0801A16F610EA26F000EA36FFEEC78
:104822000FF069C49FF86AC4A0F845EC13F0080EB3
:10483200916F010E926F030E936FE7EC1BF0100E57
:10484200916F010E926F010E936FE7EC1BF0200E39
:10485200916F010E926F020E936FE7EC1BF0140E34
:10486200916F000E926FBBEC1DF0F0EC1DF069C46D
:104872009FF86AC4A0F88D0E0801A16F620EA26FA4
:10488200000EA36FFEEC0FF069C49FF86AC4A0F893
:1048920045EC13F0DBEC12F0FF0E0801916FA3EC74
:1048A20015F0140E916F000E926FBBEC1DF0F0EC40
:1048B2001DF09D8AF28E89808992D5EC15F0D6EC96
:1048C20014F08970D5EC15F0D6EC14F0800E0801C6
:1048D200916F0F0E926F020E936F05EC14F0800E23
:1048E200916F0F0E926F020E936FCC0E946F30EC9D
:1048F20014F0800E916F0F0E926F020E936F440EA2
:10490200946F30EC14F066EC14F0800E916F0F0E81
:10491200926F020E936F05EC14F0800E916F0F0EE2
:10492200926F020E936FCC0E946F30EC14F0800EE7
:10493200916F0F0E926F020E936FBE0E946F30EC5A
:1049420014F0130E0B6E440E0C6E440E0D6E0D2EF3
:10495200FED70C2EFCD70B2EFAD70000800E916FDB
:104962000F0E926F020E936F60EC13F000C01BF4F7
:10497200000E04011C6F800E0801916F0F0E926FE2
:10498200020E936F60EC13F000C003F0026A0401A0
:104992001B510224006E1C510320016E00C04EF414
:1049A20001C04FF400C091F801C092F894EC1CF0E1
:1049B20000C0ADF6EC0E08019F6F070EA06F19EC58
:1049C20012F0EC0E9F6F070EA06FD7EC10F000C034
:1049D200AFF601C0B0F6020E005C026E000E015886
:1049E200036EEC0E0224E96E070E0320EA6E300E0F
:1049F200EE5C036E03C004F00436049004360490A7
:104A02000436049004360490010E005C026E000E1F
:104A12000158036EEC0E0224E96E070E0320EA6EC3
:104A2200300EEE5C026E025004240601AE6F050EDB
:104A3200005C026E000E0158036EEC0E0224E96E59
:104A4200070E0320EA6E300EEE5C046E04C002F024
:104A5200023602900236029002360290023602902C
:104A6200040E005E000E015AEC0E0024E96E070EE1
:104A72000120EA6E300EEE5C006E00500224B26F2E
:104A8200B70E08019F6F060EA06FF50EA16F620EA2
:104A9200A26F000EA36FFEEC0FF0C00E0801916F23
:104AA200060E926FEC0E936F070E946F010E0601C5
:104AB200AF5D0801956F000E0601B0590801966FAF
:104AC2005FEC15F0B70E9F6F060EA06F45EC13F06A
:104AD200DBEC12F0270E0601C66FE00E08019F6F95
:104AE200600EA06F000EA16FF8EC11F08972E7EC76
:104AF2000FF00B0E0401526F000E536F190E0B6E66
:104B02005A0E0C6EB10E0D6E0D2EFED70C2EFCD76A
:104B12000B2EFAD700000000000E06010F1902E169
:104B2200000E0E1904E108014EB301D0F5D7000EB4
:104B320006010F1902E1010E0E19D8A488D008014E
:104B42004EB385D0F29A83B615D083B413D07E0EBD
:104B52009F6F600EA06F000EA16FC6EC0FF00501F3
:104B6200BF6B0E0E08019F6F050EA06FA7EC10F031
:104B72004EEC10F0EC0E08019F6F070EA06F190E9D
:104B8200A16F640EA26F000EA36FFEEC0FF00E0E6B
:104B92000801916F050E926FEC0E936F070E946FE2
:104BA20014EC16F000C0B3F601C0B4F6000E026EAB
:104BB2000150025C02E1005000083FE208018E6BE6
:104BC2008F6B000E8F5D02E15F0E8E5D15E21C0E93
:104BD2008E25E16E060E8F21E26E8E510601B325FF
:104BE200E96E08018F510601B421EA6EEECFE6FFAD
:104BF20008018E4B8F2BE5D75F0E0601B325E16EC0
:104C0200000EB421E26EE66A95EC17F000C050F493
:104C120001C051F4000E011802E10A0E00180DE164
:104C220072EC19F00A0E0801916F050E926F54ECA6
:104C320016F000C0B5F601C0B6F60801270E9F6F48
:104C4200640EA06F000EA16FF8EC11F012D09F0E4F
:104C520008019F6F600EA06F000EA16FF8EC11F0BB
:104C6200530E08019F6F610EA06F000EA16FC6EC7C
:104C72000FF06B0E0401696F040E6A6F010E0601DC
:104C8200AB15016EACC602F0000E0216000E021841
:104C920002E1000E011829E169C49FF86AC4A0F874
:104CA200780E0801A16F620EA26F000EA36FFEECD8
:104CB2000FF0ABC69FF8ACC6A0F80C0E0401692534
:104CC2000801A16F000E04016A210801A26F51ECD4
:104CD20012F0010E916F926B69C493F86AC494F852
:104CE200010E956F52EC1EF00CD00801010E916F6F
:104CF200926BB70E936F060E946F010E956F52EC86
:104D02001EF06B0E0401696F040E6A6F69C49FF88E
:104D12006AC4A0F80D0E0801A16F620EA26F000E08
:104D2200A36FFEEC0FF0070E0401692508019F6FC7
:104D3200000E04016A210801A06FDC0EA16F060EAD
:104D4200A26F27EC10F069C49FF86AC4A0F8D7ECF0
:104D520010F000C0AFF601C0B0F6000E015C02E137
:104D6200140E005C0CE20601AF5104016925E16EEC
:104D72000601B05104016A21E26E200EE66E010EB8
:104D82000801916F010E926F69C493F86AC494F896
:104D9200010E956F52EC1EF06B0E0401696F040E4A
:104DA2006A6F69C49FF86AC4A0F8F70E0801A16F80
:104DB200610EA26F000EA36FFEEC0FF0070E04014E
:104DC200692508019F6F000E04016A210801A06F86
:104DD200740EA16F080EA26F27EC10F069C49FF841
:104DE2006AC4A0F8D7EC10F000C0AFF601C0B0F66C
:104DF200000E015C02E1140E005C0CE20601AF51F0
:104E020004016925E16E0601B05104016A21E26ED6
:104E1200200EE66E010E0801916F020E926F69C4B8
:104E220093F86AC494F8010E956F52EC1EF06B0E63
:104E32000401696F040E6A6F69C49FF86AC4A0F81E
:104E4200E10E0801A16F610EA26F000EA36FFEECCE
:104E52000FF0070E0401692508019F6F000E04017F
:104E62006A210801A06FFA0EA16F040EA26F27EC4F
:104E720010F069C49FF86AC4A0F8D7EC10F000C023
:104E8200AFF601C0B0F6000E015C02E1140E005C48
:104E92000CE20601AF5104016925E16E0601B05131
:104EA20004016A21E26E200EE66E010E0801916F86
:104EB200030E926F69C493F86AC494F8010E956F59
:104EC20052EC1EF00601AB4BAC2B83B60AD00801A4
:104ED2004E85530E9F6F080EA06F45EC13F0DBEC6E
:104EE20012F083B402D008014E950801000E4D194C
:104EF20002E1010E4C1913E1630E9F6F620EA06F67
:104F0200000EA16FC6EC0FF007012C6BEC0E08012E
:104F12009F6F060EA06FA7EC10F0D5EC15F0D1D460
:024F2200FFD7B7
:10643E0010EE19F0430E006E050E016E140EF66E80
:0E644E00550EF76E000EF86E70EC14F0120092
:104F2400000000000000000000000000000000007D
:104F3400000000F800000000000000333000000012
:104F440000100C06100C0600000000000000000019
:104F540040C07840C0784000043F04043F0404008B
:104F6400007088FC08300000001820FF211E00009B
:104F7400F008F000E018000000211C031E211E00B0
:104F840000F00888700000001E2123241927211036
:104F940010160E00000000000000000000000000D9
:104FA400000000E018040200000000071820400080
:104FB40000020418E0000000004020180700000070
:104FC400404080F0804040000202010F01020200D4
:104FD400000000F0000000000101011F01010100B8
:104FE400000000000000000080B07000000000001D
:104FF40000000000000000000001010101010101A6
:10500400000000000000000000303000000000003C
:105014000000000080601804006018060100000011
:1050240000E010080810E000000F102020100F000E
:10503400001010F8000000000020203F2020000095
:1050440000700808088870000030282422213000ED
:1050540000300888884830000018202020110E00F5
:105064000000C02010F8000000070424243F24009E
:1050740000F80888880808000019212020110E0073
:1050840000E0108888180000000F112020110E0085
:1050940000380808C83808000000003F000000007D
:1050A4000070880808887000001C222121221C003E
:1050B40000E010080810E0000000312222110F0067
:1050C400000000C0C00000000000003030000000FC
:1050D400000000800000000000008060000000006C
:1050E4000000804020100800000102040810200085
:1050F40040404040404040000404040404040400D0
:105104000008102040800000002010080402010064
:10511400007048080808F000000000303601000064
:10512400C030C828E810E0000718272423140B0017
:105134000000C038E0000000203C23020227382091
:1051440008F8888888700000203F202020110E0075
:10515400C03008080808380007182020201008006C
:1051640008F808080810E000203F202020100F0055
:1051740008F88888E8081000203F20202320180021
:1051840008F88888E8081000203F20000300000089
:10519400C03008080838000007182020221E02002A
:1051A40008F808000008F808203F210101213F20E9
:1051B400000808F8080800000020203F2020000014
:1051C40000000808F8080800C08080807F00000004
:1051D40008F888C028180800203F2001263820003D
:1051E40008F8080000000000203F202020203000A4
:1051F40008F8F800F8F80800203F003F003F2000BE
:1052040008F830C00008F808203F200007183F00C5
:10521400E01008080810E0000F10202020100F00F4
:1052240008F808080808F000203F210101010000E7
:10523400E01008080810E0000F18242438504F002C
:1052440008F8888888887000203F2000030C3020EC
:1052540000708808080838000038202121221C002A
:10526400180808F8080818000000203F2000000073
:1052740008F808000008F808001F202020201F005C
:105284000878880000C83808000007380E010000BC
:10529400F80800F80008F800033C0700073C030086
:1052A400081868808068180820302C03032C3020EC
:1052B4000838C800C83808000000203F200000005B
:1052C40010080808C83808002038262120201800B3
:1052D400000000FE020202000000007F4040400087
:1052E400000C30C000000000000000010638C000BF
:1052F40000020202FE000000004040407F00000067
:10530400000004020202040000000000000000008B
:105314000000000000000000808080808080808089
:105324000002020400000000000000000000000071
:1053340000008080808000000019242222223F2067
:1053440008F8008080000000003F112020110E00AA
:105354000000008080800000000E11202020110039
:10536400000000808088F800000E112020103F20EB
:105374000000808080800000001F2222222213006F
:10538400008080F0888888180020203F20200000BA
:105394000000808080808000006B9494949360006F
:1053A40008F8008080800000203F210000203F207A
:1053B40000809898000000000020203F202000007A
:1053C400000000809898000000C08080807F00006A
:1053D40008F8000080808000203F24022D30200047
:1053E400000808F8000000000020203F20200000F2
:1053F4008080808080808000203F20003F20003F0C
:105404008080008080800000203F210000203F2019
:105414000000808080800000001F202020201F00CA
:10542400808000808000000080FFA12020110E00F9
:105434000000008080808000000E112020A0FF80EA
:10544400808080008080800020203F212000010097
:1054540000008080808080000033242424241900EC
:10546400008080E0808000000000001F20200000F9
:105474008080000000808000001F202020103F203A
:10548400808080000080808000010E3008060100CA
:1054940080800080008080800F300C030C300F006F
:1054A40000808000808080000020312E0E3120009A
:1054B400808080000080808080818E7018060100CA
:1054C40000808080808080000021302C22213000E8
:1054D40000000000807C020200000000003F404009
:1054E40000000000FF00000000000000FF000000BA
:1054F4000002027C800000000040403F00000000E9
:105504000006010102020404000000000000000083
:105514000003050911FF118905C300E000F000F83C
:10552400000000000000004428FF11AA440000000D
:105534000000000000000000000000000000000067
:105544000000000000000000000000000000000057
:105554000000000000000000000000000000000047
:105564000000000000000000000083013844829223
:1055740092740183000000000000007C44C7017D98
:105584007D7D7D017D7D7D7D017D7D7D7D01FF00B6
:105594000000000000010001000100010001000101
:1055A40000000000000000000001010000000000F5
:1055B40000000000000000000000000000000000E7
:1055C40000000000000000000000000000000000D7
:1055D40000000000000000000000000000000000C7
:1055E40000000000000000000000010100000000B5
:1055F40000000101000000000000000000010101A2
:105604000101010101010101010101010101010087
:105614000000000000000000004040404040000046
:105624006D6D6D6D6D0000606060606000004040F5
:1056340040404000000000000000000000000000A6
:105644000000000000000000000000000000000056
:105654000000000000000000000000000000000046
:105664000000000000000000000000000000000036
:105674000000000000000000000000000000000026
:105684000000000000000000000000000000000016
:10569400000000000000000000DBDBDBDBDB0000BF
:1056A400DBDBDBDBDB0000DBDBDBDBDB0000DBDBB2
:1056B400DBDBDB0000DADADADADA0000D8D8D8D8B3
:1056C400D80000C0C0C0C0C00000C0C0C0C0C0007E
:1056D40000C0C0C0C0C00000C0C0C0C0C0000080C6
:1056E40080808080000000000000000000000000B6
:1056F40000000000000000000000000000000000A6
:105704000000000000000000000000000000000095
:105714000000000000000000000606060606000067
:10572400060606060600000606060606000006062D
:105734000606060000060606E6662000060686063D
:105744000600000606060686000006060606060093
:1057540000868686868680808686068686C0C08683
:1057640086860606D030760606060600000606067D
:1057740006060000060606060600000606060606DD
:1057840000000606060606000000000000000000F7
:105794000000000000000000000000000000000005
:1057A40000000000000000000000000000000000F5
:1057B40000000000000000000000601C00FE00016A
:1057C4000200C41820029E63B20E00FF8181FF0014
:1057D400008040300F00000000FF0023EAAABFAAA7
:1057E400EA033F00FF00000000000000000000008A
:1057F40000000000000000000000000000000000A5
:105804000000000000000000000000000000000094
:105814000000008080800000000000808080000084
:105824000000000000000000000000000000000074
:1058340000000000000000000E0C0800000101013F
:1058440001010000000100000001008180808180CE
:1058540081808080800101010100000001000000BE
:1058640001000101090C0E0000000000000000000E
:105874000000000000000000C0C0C0C0C0C0C0C024
:10588400C0C0C0C0C0C0C0C0C0C0C0C0C0C0C000D4
:10589400001E21404050215E001E21404050215EE8
:1058A40000000000000000000000000000000000F4
:1058B40000000000000000000000000000000000E4
:1058C4000000000000000000000000FFFFC1C1FF55
:1058D400FFC1C1FFFF000000000000000000000045
:1058E40000000000000000000000000000000000B4
:1058F4000000000000000000FFFF80FCF3EFF3FC59
:1059040080FF80EEEEEEF5FBFF9CBEB6B688FF008E
:02591400000091
:0259160000008F
:10591800625E00525F00825F00B25F00225F009209
:105928005E00C25E00F25E00325E00025E00D25D82
:01593800006E
:04593900000000006A
:0C593D00DC63000464000B6400E4630001
:0259490000005C
:02594B0000005A
:02594D00060052
:04594F000000000054
:025953002C0026
:025955002C0024
:105957000000000000000000002F0000000007000A
:10596700070000147F147F1400242A7F2A12006284
:10597700640813230036495522500F090F09000008
:1059870000001C224100000041221C000014083EB8
:1059970008140008083E0808000000A0600000087E
:1059A70008080808000060600000002010080402D2
:1059B700003E5149453E0000427F40000042615190
:1059C7004946002141454B31001814127F1000272A
:1059D70045454539003C4A494930000171090503ED
:1059E70000364949493600064949291E000036361E
:1059F7000000000056360000000814224100001481
:105A0700141414140000412214080002015109065D
:105A170000324959513E007C1211127C007F4949DE
:105A27004936003E41414122007F4141221C007F0F
:105A370049494941007F09090901003E4149497A1D
:105A4700007F0808087F0000417F41000020404197
:105A57003F01007F08142241007F40404040007F03
:105A6700020C027F007F0408107F003E4141413E47
:105A7700007F09090906003E4151215E007F09198F
:105A870029460046494949310001017F0101003F8C
:105A97004040403F001F2040201F003F4038403F0C
:105AA7000063140814630007087008070061514970
:105AB700454300007F414100000204081020000018
:105AC70041417F0000040201020400404040404081
:105AD700000001020400002054545478007F484419
:105AE700443800384444442000384444487F003850
:105AF7005454541800087E0901020018A4A4A47C79
:105B0700007F080404780000447D40000040808442
:105B17007D00007F102844000000417F4000007C8A
:105B270004180478007C0804047800384444443896
:105B370000FC242424180018242418FC007C0804E2
:105B4700040800485454542000043F444020003CBB
:105B57004040207C001C2040201C003C4030403C42
:105B6700004428102844001CA0A0A07C00446454D2
:085B77004C441414141414141E
:105B7F002048617264773A202050494320436C6972
:105B8F00636B65722031384634374A3533200D0A3E
:105B9F00204F6C65642053534431333036203132FB
:105BAF003878333220302E3936200D0A20445331C5
:105BBF00384232302073656E736F72200D0A2047A2
:105BCF0050532055426C6F7820374E200D0A2055C8
:0A5BDF0041525432200D0A0D0A0055
:105BE90020446F73736965723A433A5C5F4D696B20
:105BF900726F435C5F4D657350726F6A6574735F52
:105C09004D696B726F435C5F31384634374A3533BF
:105C19005F4750535F55415254315F554152543299
:105C29005F445331384232305F4F4C45440D0A00CE
:105C390020536F75726365203A20436C69636B6505
:105C4900725F31384634374A35335F5541525431E2
:105C59005F4F6C65645F535344313330365F44534F
:105C690031384232305F475053374E5F55415254B5
:0D5C7900325F3139303830352E630D0A00AE
:105C860020417574726573203A20204F4C45445F5D
:105C9600493243325F3139303830312E63202C207F
:105CA6004F4C45445F4932435F3139303830312EED
:105CB60068202C204F4C45445F5461626C65735FCD
:0B5CC600313930382E680D0A0D0A003D
:105CD10033206C69676E6573206465203230206300
:105CE100617273204142434445464748494A4B4CFF
:105CF1004D4E4F505152535455565758595A206191
:105D010062636465666768696A6B6C6D6E6F7071FA
:085D1100727374757677780057
:105D190020496E666F7320616666696368E9657319
:105D290020766961205541525431206D6F64756C3C
:105D3900E9657320656E20666F6E6374696F6E2006
:105D4900646520425031206574204250320D0A00AA
:105D5900205541525432206D617070656420313292
:105D690030302C382C4E2C312054582070696E203C
:105D79005244362D52503232202C205278207069EC
:0D5D89006E205244352D525032330D0A0069
:105D96002050726F6A65743A436C69636B65725F13
:105DA60031384634374A35335F4F6C65645F475048
:105DB600535F445331384232305F484331325F31AA
:0C5DC6003930382E6D637070690D0A00D2
:105DD20000000000000000000000000000000000C1
:105DE20000000000000000000000000000000000B1
:105DF20000000000000000000000FFFFFFFF0000A5
:105E020000E0F8FCFEFF1F0F0F0F1FFEFEFCF080EC
:105E120000070F3F3F7F7C7878783CFFFFFFFFFF52
:105E2200000E3E7E7EFEF8F0F0F07C7F3F1F0F01F9
:105E320000F0FCFEFEFF1F0F0F0F1FFFFEFEFCF027
:105E42000081C3E7FFFF7E3C3C3C7EFFFFE7C3814E
:105E5200000F3F7F7FFFF8F0F0F0F8FF7F7F3F0FEA
:105E62000080F0FCFEFE3F0F0F0F3FFEFEFCF080B5
:105E720000FFFFFFFFFF0000000000FFFFFFFFFF2A
:105E820000030F3F7F7FFCF0F0F0FC7F7F3F0F01AC
:105E9200000080FCFFFFFF3F1F1F1F1F1F1F1F006F
:105EA20000183F3F3F3F1F0F0F0F1FFFFEFEF8E09E
:105EB20000061F3F7F7FFCF0F0F0F87F7F3F1F0757
:105EC2000080F0F8FCFE3E0F0F0F1F7F7E7E7C707D
:105ED20000FFFFFFFFFF3C1E1E1E3EFEFCFCF0E02B
:105EE20000010F3F7F7FF8F0F0F0F8FF7F3F1F07C0
:105EF200001F1F1F1F1F1F1F1F9FFFFFFF3F1F0F9F
:105F02000000000000E0F8FCFF7F0F03000000002B
:105F1200000000F0FFFFFFFF07000000000000008C
:105F22000000000000C0E0F8FCFFFFFFFFFF0000E0
:105F3200C0E0F8FCFFBF8F8381FFFFFFFFFF80807F
:105F4200070707070707070707FFFFFFFFFF070707
:105F5200000000C0E0E0F0F87CFEFFFFFFFF000061
:105F6200000000030101000000FFFFFFFFFF00002F
:105F7200000000000000000000FFFFFFFFFF000024
:105F820000E0F8FCFEFE1F0F0F0F1FFFFEFEFCF0ED
:105F9200000000000080C0E0F0F8FE7F3F1F070114
:105FA20000C0F8FCFFFFFFFFF9F9F8F8F8F8F8F87D
:105FB2000030787E7E7F1F0F0F1FFFFEFEFCF00079
:105FC200000000000000000E0E0F1FFBFBF9F0C0E6
:105FD20000061F3F7F7FFCF0F0F0FC7F7F3F1F0732
:105FE20020554152543220393630302C382C4E2C28
:105FF200312054582070696E20524336202C205292
:0C600200782070696E205243370D0A00B0
:10600E00204275732049324320706F7572204563AC
:10601E0072616E204F4C4544205353443133303619
:0A602E00203132387833320D0A00B9
:10603800205465737420536F6E6465204F57532046
:106048004453313842323020737572205241322025
:036058000D0A002E
:10605B000D0A4B6579626F61726420546F756368CA
:10606B00205541525431206F722054696D656F7504
:03607B007420008E
:10607E00526563657074696F6E2073757220554139
:10608E00525432205258203D20475053203A0D0A88
:01609E000001
:10609F002042414420526563657074696F6E206FB2
:1060AF0075204465636F64616765204747410D0A3A
:0160BF0000E0
:1060C000206F752034206C69676E657320646520CD
:1060D000323020636172732036783870200D0A00E8
:1060E0002055415254322C2077616974696E6720C3
:0D60F000475053206461746173203A200012
:1060FD00204D435520203A2031384634374A353328
:0D610D005F51464E5F343470696E0D0A001C
:10611A0020524431202D2D3E2049324332202D2D4C
:0D612A003E534441204F4C4544200D0A00D7
:1061370020524430202D2D3E2049324332202D3E1F
:0C6147002053434C204F4C45440D0A00EF
:10615300204D61757661697365205265636570745E
:0A616300696F6E204750530D0A00CB
:10616D002041666669636865203320636172732020
:09617D00537065636961757800D7
:10618600204F4C4544204C4344204E6F6E20747281
:086196006F7576E9200D0A0087
:10619E0020506F77657220737570706C793A20336A
:0761AE002C3320560D0A00FE
:1061B500426967204D73672064652036302063612E
:0661C5007273203A200075
:1061CB0020323020436861727320737572204C69E2
:0661DB00676E6520310033
:1061E10020416C74693A202020202020202020208A
:0661F10020202020200008
:1061F700204C6174693A2020202020202020202074
:06620700202020202000F1
:10620D00204C6F6E673A2020202020202020202057
:06621D00202020202000DB
:106223004932433220696E69742061742031303001
:066233004B687A0D0A0021
:10623900203720204269672043617273202031365C
:05624900783136200051
:10624E0031323334353637383930313233343536FE
:05625E00373839300063
:10626300526563752064652055415254312052585C
:05627300203A2020008C
:1062780020426F75636C6520232020202020202079
:05628800202020200091
:10628D00204F6C65642046494C4C2077697468201A
:05629D003078464600C8
:1062A2004D73672031342063617273207461696CAD
:0562B2006C65203200C4
:1062B7003132333435362D4142432D6162632D36F9
:0562C7003738393000FA
:1062CC004C34204E554D42455253203031323334EC
:0562DC003536373800E3
:1062E1004D7367207375722034656D204C69676E3C
:0462F1006520200004
:1062F5002054656D7065723D20202020202020B03F
:02630500430053
:10630700204D657375726520445331384232303DF4
:02631700200064
:10631900436865636B2044657669636520402000A6
:106329002046616D696C7920436F6465203A2000CD
:1063390030313233343536373839414243444546B2
:0F6349000D0A204F4C454420696E69740D0A00FF
:0E635800206973206E6F7420666F756E64008E
:0D6366002078203130306D7365630D0A0022
:0D637300204F4C454420696E69740D0A00EE
:0C6380002020202020416C74203A2000D6
:0C638C002020202048444F50203A2000E0
:0B639800202020536174656C3A200047
:0B63A300204F4C4544204F4E0D0A00D7
:0A63AE00202020204669783A2000E4
:0A63B80020666F756E64204F4B00E5
:0963C200322020484152445700EA
:0963CB0020204C6174203A2000EE
:0863D400204C6F6E203A2000FE
:0863DC0000007E66667E0000F1
:0863E4000F090F00000000008A
:0863EC00206F6E2049324300CE
:0863F40020204352433D20002C
:0863FC0020494431203D20003E
:07640400C030383E38306063
:07640B00060C1C7C1C0C06B2
:076412004B4D4C203A200025
:0764190024475047474100F2
:076420003132342E39360041
:06642700204F4B0D0A009E
:05642D00B04320200037
:04643200205A2000CC
:0464360020592000C9
:04643A0020582000C6
:020000040001F9
:08FFF800ACF7FCFFFFFBFFFB6F
:00000001FF
